:104BD8007584008539D2853AD3758401853BD285A1
:104BE8003CD3E4F53AF5393000733056688566826F
:104BF800856583E0F5691281D7E56C2539F539E5D6
:104C08006B353AF53AA3858266858365E565656304
:104C1800700AE56665647004D2668041E565641FC4
:104C2800700CE56664FF700675660075650430589B
:104C38002C856482856383E56AF0A3858264858315
:104C480063E563641F7016E56464FF7010756400A3
:104C58007563048008853E3A853D39800030010C33
:104C6800E539253FF539E53A3540F53A300206E5AC
:104C780033253AF53A300310E50A8536F0A425398C
:104C8800F539E5F0353AF53A300410E5118535F097
:104C9800A42539F539E5F0353AF53AE4F53CF53B24
:104CA80030080D200908853E3C853D3B8002800088
:104CB800300A0CE53B253FF53BE53C3540F53C30FB
:104CC8000B06E533253CF53C300C10E50A8536F03B
:104CD800A4253BF53BE5F0353CF53C300D10E511DE
:104CE8008535F0A4253BF53BE5F0353CF53C2290B5
:104CF8004D3A302903124D07302A03124D1722E589
:0E4D08000B2509F50BE50C3508F50C93F50AA3
:104D160022E512250EF512E513350DF51393C3138F
:104D2600F8E5142510F514E515350FF51593C3139D
:104D360028F511227F8285888C8F9295989B9EA15B
:104D4600A4A7AAADB0B3B6B9BBBEC1C3C6C9CBCEC4
:104D5600D0D3D5D7D9DCDEE0E2E4E6E7E9EBEDEE49
:104D6600F0F1F2F4F5F6F7F8F9FAFBFCFCFDFDFEBE
:104D7600FEFEFEFEFEFEFEFEFEFDFDFCFCFBFAFA5E
:104D8600F9F8F7F6F4F3F2F0EFEDECEAE8E7E5E32D
:104D9600E1DFDDDBD8D6D4D1CFCDCAC8C5C2C0BD10
:104DA600BAB7B4B2AFACA9A6A3A09D9A9794908DBA
:104DB6008A8784817E7A7774716E6B6865625F5CC0
:104DC600595653504D4A4744423F3C393734322FA7
:104DD6002D2A282624211F1D1B1918161412110FFF
:104DE6000E0C0B0A08070605040403020201010063
:104DF600000000000000000000010102020304059B
:104E0600060708090A0B0D0E1011131516181A1CA1
:104E16001E20222427292B2E303335383A3D404296
:104E260045484B4E515456595C606366696C6F72C7
:104E360075787B7FE537F5F0753D00E53EC3945602
:104E46004013A4F5F0C394565007E5F02456F53EFA
:104E560022753EAC227456953EA4F8C3945650066D
:104E6600745698F53E22753E0022E538F5F0B401F9
:104E76000122753F00E540C394704020200907B425
:104E8600010475407022A420D20EF5F0C394705030
:104E960007E5F02470F540227540FF22C374709533
:104EA60040200907B4010475407022A4F820D20BF3
:0F4EB600C394705006747098F540227540002226
:107C4800D2F4C2F5C2F675840F85F0C81253A67433
:107C580003127C971253967403127C971253851261
:107C680053857403127C971253857402127C971201
:107C780053857428127D067406127D06740E127DD3
:107C8800067401127D061253967480127D0622C076
:107C980000A2E092F3A2E192F2A2E292F1A2E392B0
:107CA800F0D2F475840F85F0C8C2F47830D8FE8518
:107CB800F0C87830D8FED00022C00075840FA2E446
:107CC80092F3A2E592F2A2E692F1A2E792F0D2F440
:107CD80085F0C8C2F47830D8FE85F0C87830D8FE70
:107CE800D00022203817EF75840FD2F5C2F685F040
:107CF800C8127CC1125385127C9712538522758451
:107D08000FC2F5C2F685F0C8127CC1125385127CE9
:107D1800971253852220380DEF14A2E492E6C2E4AC
:107D2800D2E7127D0622740F127D0622740D127D91
:107D3800062220380E7F01127D1D78107F20127CCC
:107D4800EBD8F92220380E7F11127D1D78107F2084
:067D5800127CEBD8F922B9
:10754C00C2B6758400D2C2C2C6D2C6C2C4D2C5C22B
:10755C00C330C3FD74A0F5C2C2C5C2C330C3FD8E17
:10756C00C2C2C330C3FD8FC2C2C330C3FD8DC2C201
:10757C00C330C3FDD2C4C2C320C4FD125396D2B6CD
:10758C0022758400C2C3D2C530C3FD74A0F5C2C23B
:10759C00C5C2C330C3FD8EC2C2C330C3FD8FC2C2CD
:1075AC00C330C3FDC2C4D2C5C2C330C3FD74A1F580
:1075BC00C2C2C5C2C330C3FDC2C2C2C330C3FD8583
:1075CC00C207D2C4C2C320C4FD22D2C2C2C6D2C614
:1075DC00D2C4C2C320C4FD22758400D2C2C2C6D29A
:1075EC00C6C2C4D2C5C2C330C3FD74A0F5C2C2C5E5
:1075FC00C2C330C3FD8EC2C2C330C3FD8FC2C2C36F
:10760C0030C3FD8C838D827B40E0A3F5C2C2C330B6
:10761C00C3FDDBF5D2C4C2C320C4FD125396227540
:10762C008400C2C3D2C530C3FD74A0F5C2C2C5C2AA
:10763C00C330C3FD8EC2C2C330C3FD8FC2C2C330C0
:10764C00C3FDC2C4D2C5C2C330C3FD74A1F5C2C24E
:10765C00C5C2C330C3FD8C838D82C2C330C3FDE56C
:10766C00C2F0A31BBB01F3C2C2C2C330C3FDE5C24F
:09767C00F0D2C4C2C320C4FD22F7
:050003000248913200EB
:04000B00024BC532AD
:1054F90075FF0775FFDE75FFAD75840F75E10775DB
:10550900E20475E34475840F75A43575A50975A67C
:10551900BB75A7FF759CFF759D00759E00759FF073
:1055290075D8FF75E8FF75F80F75AD0F75840175AE
:10553900893075888F75840275893075888F75846F
:105549000F758A80758C67780874FF000000000069
:1055590000000000000000D5E0F1D8EDE58C30E74F
:10556900FB759701758A0043890475840075B71026
:1055790075840F438901758D02758F01758E0474C9
:1055890080D5E0FD438902E58930E4FB7597027512
:10559900840075D10775840075BB0175BA0075BCA7
:1055A900F075C70075C60075C5FF75C4FF75E8813C
:1055B90075840275BB0475BA0075BCF175C60075B2
:1055C900C4FF75E88875840075D48475840175D421
:1055D90084758400C2F8759A47759D1A43F8097550
:1055E900870075840075B90075A9007591007598D3
:1055F9005075840175989075840075C04075C30015
:1056090075CFF2758400758E1075892175880575B9
:105619008400758A00758BE0758CF4758DE043887C
:105629004075840075C90075CA0075CB0075CC003A
:1056390075CD0075840175C91875CA8075CBFB7560
:10564900CDFB75CC80D2CA75840275C91875CAA6F6
:1056590075CBAF75CDAF75CCA6D2CA75840075EF81
:105669000275A8AC75B81D75E6B075E71775F60033
:1056790075F74378A0760A76A1780A78A276067536
:07568900A8859000007F00DE
:105690007E20E4F0A3DFFCDEFA7534327535FF7549
:1056A00036C878A0760A78A1760A78A27606D2B6AD
:0456B0001275D62277
:10531B0075840FD2FD2275840FC2FD2275840FD2C6
:10532B00FC2275840FC2FC2275840FD2FED234226C
:10533B0075840FC234C2FE22C29322D2932275848B
:10534B000FA2FA2275840FA2F92275840FA2DD2217
:10535B00A2922275840FA2DA2275840FA2DB22752A
:10536B00840FA2D82275840FA2D92200000000005E
:10537B0000000000000000000022C000C001790402
:10538B0078B4D8FED9FAD001D00022C000C0E078A2
:10539B009C7605E670FDD0E0D00022C000C0E0781E
:1053AB009C760FE670FDD0E0D00022C000C0E07804
:1053BB009C7664E670FDD0E0D00022EF75F064843B
:1053CB0024309000CBF0E5F0A375F00A842430F084
:1053DB00A3E5F02430F022EF75F0648424309000C4
:1053EB00CBF0E5F0A375F00A842430F0A3E5F024AC
:1053FB0030F09000CBE0B4300B7420F0A3E0B4306D
:10540B00037420F022900021E0540FFFA3E0B4209E
:01541B00028E
:10541C008019540FCF75F00AA42FFFA3E0B420021B
:10542C008009540FCF75F00AA42FFF22C006C005C7
:10543C00C004900021E0540FFFFEA3E0B42003C38E
:10544C00802C540FFDCF75F00AA42FFFA3E0B420DD
:10545C0003C3801A540FFCEE75F064A420D20EFE28
:10546C00ED75F00AA42E40052C40028001D3D00427
:10547C00D005D0062275F06484F6E5F00875F00AC4
:10548C0084F608A6F008229000D1E075F009A42F4C
:10549C00FFE5F03EFE79007A537B097C008E838F0A
:1054AC0082EC9389838A82F0A3A983AA820CDBED18
:1054BC0022900057E0601775F010A42FF9EE35F02C
:1054CC00FA7BFFC006C00712ABA6D007D00690002F
:1054DC0058E0600F75F010A42FF9EE35F0FA7BFF51
:0D54EC0012A5CC2285060722228505062286
:1000A600564F4950205441424C4520424547494EFF
:1000B60000564F4950205441424C452057524F4E0E
:1000C600470020564F4950205441424C4520454E4A
:1000D6004420002020202020202020202020202016
:1000E6002020205245504541544552204E554D4200
:1000F6004552202020202020202020203120746FEF
:10010600203230202053495445204E554D42455209
:100116002020202020202020202020203120746F25
:1001260020393982020011010215011482020111DF
:1001360003041501632020202020202020202020D9
:1001460020202020202020202020202020202020A9
:10015600202020202020434F5552544553592042F9
:100166004545502020204354435353204F4E2048AA
:10017600414E47202020205553455220454E4142AE
:100186004C452020202020524553455256452054A8
:100196004F4E45202020204E4554574F524B204D60
:1001A6004F44452020204E4554574F524B204E5524
:1001B6004D42455220202020202020202020202093
:1001C6002020202020202020202020202020202029
:1001D6002020202020202020202020202020202019
:1001E6002020202020202020202020202020202009
:1001F60020202020202020202020202020202020F9
:1002060020313D454E202020202020202020202067
:10021600204D4F4445202020202020202020202033
:1002260020544F4E4564010011020C150001640272
:100236000011030C15000164040011040C150001E3
:1002460064080011050C15000164100011060D1557
:100256000002C8030111070A1901012020202020ED
:100266002020202020202020202020202020202088
:10027600202020202020202020202020434F5552BF
:10028600544553592042454550202020435443535A
:1002960053204F4E2048414E47202020205553459D
:1002A6005220454E41424C452020202020524553A5
:1002B6004552564520544F4E45202020204E455449
:1002C600574F524B204D4F44452020204E45545702
:1002D6004F524B204E554D42455220202020202083
:1002E6002020202020202020202020202020202008
:1002F60020202020202020202020202020202020F8
:1003060020202020202020202020202020202020E7
:1003160020202020202020202020202020202020D7
:1003260020202020202020313D454E202020202046
:10033600202020202020204D4F4445202020202012
:1003460020202020202020544F4E45640100110219
:100356000C15000164020011030C15000164040071
:1003660011040C15000164080011050C1500016448
:10037600100011060D150001C8030111070A190125
:100386000120202020202020202020202020202086
:100396002020202020202020202020202020202057
:1003A6002020434F5552544553592042454550202D
:1003B6002020205553455220454E41424C45202091
:1003C600202043524F535320544F4E45204D4F4407
:1003D600452043544353532F4443532043524F53D2
:1003E6005320204E4554574F524B204D4F444520E5
:1003F60020204E4554574F524B204E554D424552A4
:1004060020202020202020202020202020202020E6
:1004160020202020202020202020202020313D4583
:100426004E2020202020202020202020204D4F4418
:1004360045202020202020202020202020544F4E00
:100446004520202020202020202020202020202081
:10045600206401001102091500016402001103095C
:1004660015000164040011060A150001C8030111F4
:10047600070C1901012020202020202020202020E8
:100486002020202020202020202020202020202066
:1004960020202020200101010101010101010000AD
:1004A6000000000000000000000000000000000046
:1004B6000000000000000000000000000000000036
:1004C6000000000000000000000000000000000026
:1004D6000000000000000000000000000000000016
:1004E60000000000000000000000000000000020E6
:1004F60020202020202020202020202020202020F6
:100506002020202020202020202020202020200104
:1005160001010101010101010000000000000000CD
:1005260000000000000000000000000000000000C5
:1005360000000000000000000000000000000000B5
:1005460000000000000000000000000000000000A5
:100556000000000000000000000000000000000095
:1005660000000000000000000020202020202020A5
:100576002020202020202020202020202020202075
:10058600202020202020202020010101010101013E
:100596000101202020202020202020202020202093
:1005A6002020202020202020202020202020202045
:1005B60020202054454C434F2050524F4752414D26
:1005C600202020524144494F2050524F4752414D1E
:1005D60020202050484F4E452050524F4752414D03
:1005E600202020434F4D50552050524F4752414DE9
:1005F6002020202041434345535320434F44452068
:10060600202044544D462054454C434F204C4556DB
:10061600454C44544D4620524144494F204C455682
:10062600454C4245455020524144494F204C455681
:10063600454C424545502054454C434F204C455669
:10064600454C4357494420524144494F204C455656
:10065600454C564F49434520524144494F204C454D
:10066600564C564F4943452054454C434F204C4524
:10067600564C5041474520524144494F204C45561F
:10068600454C435443535320524144494F204C4513
:10069600564C44435320524144494F204C455645FD
:1006A6004C204C545220524144494F204C4556450B
:1006B6004C2052505420524144494F204C455645F7
:1006C6004C2054454C434F20524144494F204C4501
:1006D600564C524144494F2054454C434F204C45BB
:1006E600564C524144494F204C494D4954204C45A3
:1006F600564C20434F53204F5220535155454C439F
:1007060048202020434F5320504F4C4152495459C2
:100716002020434F53205452494747455220564FB5
:100726004C54434F53204143515549535420544947
:100736004D45434F532052454C454153452054495E
:100746004D452053454E534520504F4C4152495438
:10075600592053454E205452494747455220564F3B
:100766004C5453454E204143515549535420544906
:100776004D4553454E2052454C454153452054491D
:100786004D45204C545220484F4C442044454C4142
:100796005920505454205455524E4F4646205449E1
:1007A6004D4552455045415445522054494D454FBB
:1007B60055542020414E54492D4B45524348554EE1
:1007C6004B202020535155454C4348205441494C19
:1007D60020202043544353532F44435320484F4C27
:1007E600442043524F535320425553592044454CBD
:1007F600415943524F5353204255535920484F4C69
:10080600442020204C54522053594E4320424954F0
:10081600202020414456414E43454420204C4F431E
:100826004B20202020202020202020202020202097
:1008360020202020202020202020202020202020B2
:1008460020202020202020202020202020202020A2
:100856002020202020202020202020202020202092
:100866002020202020202020202020202020313D54
:10087600454E202020202020202020202052415498
:10088600494F2020202020202020202020303D43BA
:100896004F532020202020202020202020313D5092
:1008A6004F532020202020202020202020203120CF
:1008B6004D532020202020202020202020313020B1
:1008C6004D53202020202020202020203130302091
:1008D6004D5320202020202020202020202020537F
:1008E600454320202020202020202020313D534B2E
:1008F6004950202020202020202020202020202099
:1009060020202020202020202020202020202020E1
:100916002020205052494F52495459204C455645A3
:100926004C20204C545220454E434F444520504FB6
:100936004C20204C5452204445434F444520504FB0
:100946004C2020205445535420494420434F4445CD
:10095600202049444C45204D45535341474520549A
:100966004D5220202020415245412042495420200A
:100976002020204D4153544552204F5220534C4184
:1009860056452044435320454E434F444520504F3F
:100996004C2020444353204445434F444520504F68
:1009A6004C2020434F5552544553592044454C4101
:1009B600592020202048414E472054494D452020AB
:1009C6002020434152524945522044524F50204420
:1009D6004C5920204143434553532044454C4159EB
:1009E600202053544154494F4E204944204D4F44F2
:1009F600452020564F494345204F522043574944EE
:100A060020202020494420494E54455256414C202E
:100A16002020202020435749442053504545442058
:100A260020202043574944204652455155454E43C0
:100A36005920202043574944204D455353414745AB
:100A46002020205455524E5F4F4E2044454C41596C
:100A56002020205455524E5F4F46462044454C4177
:100A660059202042454550204652455155454E4352
:100A7600592052455045415445522044495341421C
:100A86004C45204155582052454C4159204D4F4424
:100A960045202043524F53532042555359204D4F22
:100AA6004445205245504541544552204741494E00
:100AB6002020202054454C434F204741494E2020BA
:100AC60020204E4554574F524B2048414E475449DB
:100AD6004D45202020202020202020204C45564512
:100AE6004C2020202020202020202020303D4E4F4A
:100AF600524D202020202020202020202020434F3F
:100B06004445202020202020202020202020415243
:100B160045412020202020202020303D4D415354A7
:100B26004552202020202020202020202020312057
:100B36004D5320202020202020202020203130202E
:100B46004D5320202020202020202020313030200E
:100B56004D532020202020202020202020312053EB
:100B66004543202020202020202020202031204DF9
:100B7600494E2020202020202020202020204D4FBC
:100B86004445202020202020202020303D564F495B
:100B960043452020202020202020202020204652AF
:100BA6004551202020202020202020202020313DBB
:100BB600454E2020414C41524D20434F554E542026
:100BC600202020524553544F524520434F554E54F2
:100BD6002020202020494E54455256414C202020AA
:100BE6002020204E4554574F524B20434F4445201A
:100BF6002020494E544552434F4E4E454354204DB6
:100C06004F444E4554574F524B20494E4143544949
:100C1600564582010011022D1500018201011103C2
:100C26002D15000182010211042D15000182010318
:100C360011052D150001780604110601190101821E
:100C4600030A11072E1500FF82030B11082E15004B
:100C5600FF82030C11092E1500FF82030D110A2EC7
:100C66001500FF82030E110B2E1500FF82030F11D4
:100C76000C2E1500FF820310110D2E1500FF8203A6
:100C860011110E2E1500FF820312110F2E1500FFF3
:100C960082031311102E1500FF82031411112E1555
:100CA60000FF82031511122E1500FF820316111381
:100CB6002E1500FF82031711142E1500FF8203184C
:100CC60011152E1500FF82011911162F150001822C
:100CD600011A11173015000182031B11182E150079
:100CE600FF82021C11193115006382021D111A328E
:100CF60015006382011E111B3015000182031F11AE
:100D06001C2E1500FF820220111D31150063820280
:100D160021111E32150063820222111F3315026350
:100D26008203231120321501FF8203241121341579
:100D360002FF820225112233150063820226112347
:100D460032150063820227112433150363820228B9
:100D56001125321500638203291126331500FA8204
:100D6600012A11273515000182012B11385415016E
:100D76000982012C11395515000182012D113A55B0
:100D860015000182032E113B561501FA82032F111D
:100D96003C5C1500FF820130113D571500018201B0
:100DA60031113E58150001820132113F55160001DE
:100DB60082013311405515000182023411415A1542
:100DC600006382023511425B1500638202361143CD
:100DD6005A15006382023711445A1500638201389E
:100DE60011455E15000182013911465F1500018229
:100DF600023A11475D15006382023B1148591504FA
:100E06006382023C114960150114BE0A3D114A561F
:100E1600110000820247114B5A15006382024811E5
:100E26004D60150114820149114E5E1500028201C2
:100E36004A114F6115000182014B11505E150004E5
:100E460082014C11515415010982014D115254155C
:100E5600010982024E11533415006382014F11625B
:100E66000115000982015011630115000982025122
:100E760011645D150163C8035211650115010182F4
:100E8600015311665E150002820354116734150082
:100E9600FF01010200000200000200000000000045
:100EA6000101013132333435361432320532FFFF57
:100EB600FF1919196464C8FF000180000A01800047
:100EC6000A1E1AB400001E1E1E00010000020A00BF
:100ED6000100000A1E630A000100050520202020EB
:100EE6002020202020200A05000000010114000017
:100EF600010000000044313233343536373839309A
:100F06002A2341424344AAA3C1C2C3C4D7ABA8A95A
:100F16002A23414243363330363730363934373177
:100F2600393734343737303739373832353835345E
:100F3600383835393135393438393734313030315C
:100F4600303331303731313031313431313831327B
:100F5600333132373133313133363134313134365E
:100F66003135313135363135393136323136353143
:100F76003637313731313733313737313739313821
:100F86003331383631383931393231393631393908
:100F96003230333230363231303231383232353225
:100FA600323932333332343132353032353430300F
:100FB6003630303730313530313730323130323308
:100FC60030323530323630333130333230333630FA
:100FD60034333034373035303035313035333035E1
:100FE60034303635303731303732303733303734C6
:100FF60031313431313531313631323231323531C8
:1010060033313133323133343134313134333134B5
:101016003531353231353531353631363231363591
:10102600313732313734323035323132323134328F
:101036003233323235323236323433323434323479
:101046003532343632353132353232353532363163
:10105600323633323635323636323731323734334A
:10106600303633313133313533323533333133334F
:10107600323334333334363335313335363336342D
:101086003336353337313431313431323431333428
:101096003233343331343332343435343436343510
:1010A60032343534343535343632343634343635F4
:1010B60034363635303335303635313635323335EC
:1010C60032363533323534363536353630363631D6
:1010D60032363234363237363331363332363534C9
:1010E60036363236363437303337313237323337B5
:1010F600333137333237333437343337353441428B
:10110600434445464748494A4B4C4D4E4F50515231
:10111600535455565758595A6162636465666768F1
:10112600696A6B6C6D6E6F707172737475767778B1
:10113600797A30313233343536373839607E21406A
:101146002324255E262A28295F2D2B3D7B7D5B5D8A
:101156007C3A3B3C3E2C2E3F2F2020202020202076
:10116600202020202020474C4F42414C2020202088
:1011760020202043544353533A202020202020206F
:101186002020204443533A202020202020202020C5
:1011960020202052455045415445522020202020F1
:1011A60020205350454544204449414C494E472050
:1011B600202053504545442043414C4C494E47203E
:1011C600202020505443204E554D42455220202089
:1011D600202020564F494345204D4553534147450E
:1011E600532020564F49434520504C4159424143D4
:1011F6004B202020494E56414C49442054595045D5
:10120600202020204F5554204F462052414E47451E
:10121600202020494C4C4547414C2056414C5545D1
:1012260020204D5553542046494C4C204649454CA8
:1012360044202020494C4C4547414C20434F4445CF
:1012460020202044415441204143434550544544C5
:1012560020204C494E45204E554D4245523A2020BD
:101266002020555345522050524F4752414D4D492B
:101276004E47204C54522049443A2020202020201A
:101286002020564F494345205245434F5244494E2C
:10129600472020494C4C4547414C20454E54525915
:1012A600202020494C4C4547414C2047414E472081
:1012B6002020202020434F4D504C455445442020AB
:1012C600202020474C4F42414C20454550524F4D1F
:1012D60020202020435443535320454550524F4D20
:1012E600202020202044435320454550524F4D2076
:1012F60020202020204C545220454550524F4D204E
:101306002020204449414C494E4720454550524FE4
:101316004D202043414C4C494E4720454550524FA5
:101326004D2020202050544320454550524F4D20FB
:1013360020202052455045415445522045455052A3
:101346004F4D2020494E495449414C495A494E4730
:101356002020202052455045415445523A20202015
:101366002020202020202020202020202020202077
:101376002020202020202020202020202020202067
:101386002020202020202020202020202020202057
:101396002020202020202020202020202020202047
:1013A600202020435443535320434F444520474174
:1013B6004E472044435320434F44452047414E4720
:1013C6002020205250545220434F44452047414E3E
:1013D600472020525054522047414E47202020207B
:0213E6002020C5
:107D5E0030363230350912B1E912510002AAA3129F
:107D6E00B465128A7612A0EB12A14712B35F30509F
:107D7E0005C250123CE2129F73E490022DF0900265
:107D8E002EF0C2362230372E30350512B21980321F
:107D9E0012B465128A7612A0EB12A14712B35F12CB
:107DAE009F73305005C250123CE2E490022DF090C9
:107DBE00022EF0C23722203803027E6230350612C0
:107DCE005BA802510030511A12B465128A7612A0C5
:107DDE00EB12A14712B35F129F73305005C25012BF
:107DEE003CE2E490022DF090022EF0C2382059FDB4
:107DFE00900264747EF0D2592059FD900264745042
:107E0E00F0D2592059FD9000D6E075F00A84443026
:107E1E00900264F0D2592059FD9000D6E075F00A18
:107E2E0084E5F04430900264F0D2592059FD90025E
:107E3E0064305105745DF08003745BF0D2592059A3
:107E4E00FD900264740DF0D2592059FD90026474B5
:057E5E000AF0D25922D8
:10510000900013E07012900014E0D394004009C2A4
:1051100036C237C238C23522900014E0127F3852AE
:105120003100523401523702523A03523D04523F89
:105130000552410652430752460852490A524C0B47
:10514000524F0F525210525511525814525B155271
:105150005E1652611952641A52671B526A1E526DD2
:105160001F527023527324527628527929527C2D73
:10517000527F2E52822F528530528832528B3352B8
:105180008D34529035529337529638529964529CCE
:1051900065529F6652A26752A56E52A76F52E97080
:1051A00052A97152AB7852AD7952E97A52AF7B5223
:1051B000B18252B38352E98452B58552B88C52BB46
:1051C0008D52E98E52BD8F52C09652C39752E998C4
:1051D00052C59952C8A052CBA152E9A252CEA352B5
:1051E000D1AA52D3AB52E9AC52D5AD52D8B452DBAE
:1051F000B552E9B652DEB752E0BE52E3BF52E6C046
:1052000052E9C152EBC252EEC852F1C952E9CA5238
:10521000F7CB52FAF052FDF15300F25303FA530662
:10522000FB5309FC530CFD530FFE5312FF000053B8
:105230001502B6FD02B54D02A30B02B48D800480A9
:1052400002800002A6A002620B02AEA302AFEC0233
:10525000AAE3028B2102B01F02AB220289C902B06D
:105260005202AB6102855802B08502A3B702B0B802
:1052700002A40C02B0EB02A46102B11E02B2A702AA
:10528000AE3102A6EA12A25902A1FF8000029AEFF3
:1052900002A89402999E02A08F029FD402A85002F5
:1052A000AF4B025EDE8039804880408033801C80B6
:1052B0003A8005803C02667A0286E38034026511FA
:1052C0000292CA8006026D6A028919029A800260FF
:1052D00075800D801C02639F028ED5029D08800B95
:1052E0000293DC02A604028C6D8009028208028D02
:1052F000A50296D802AD0B029A1002B2D50283B86D
:1053000002B720029C9E02001202006A020076028E
:0B5310008E3E020077E4900014F022B3
:10B6FD00E4900016F0900013741EF0900014E00416
:02B70D00F02228
:10B54D00127D3A127D4C7BFF7A12796812ABA67F81
:10B55D0011127D1DC23CC239E4900016F09000140A
:04B56D00E004F022E4
:10A30B00303952900015E0FFC239BF2A0790001474
:10A31B00E004F022BF5D0AC235E4900014F0D25184
:10A32B0022BF5B0AC235E4900014F0C25122BF2356
:10A33B00247F23127CEB900016E004F0E0C394041E
:10A34B00400DC235E4900014F0127D3A027D4C9022
:05A35B0000147402F083
:01A3600022DA
:10B48D007BFF7A12796812ABA6127D4C7F11127D6B
:10B49D001D12002EE4900050F07F2A127CEBC23C6E
:07B4AD00900014E004F022FE
:10A6A000303946900015E0F517C239E517642A6085
:10A6B00038AF1712B7605022AF17127CEB900050E2
:10A6C000E02417F582E43400F583E517F09000509C
:10A6D000E004F0900014E004F0227BFF7A127998F5
:09A6E00012ABA690001474FAF00C
:01A6E900224E
:10620B0020390302639E900015E0FFC239BF2A07B5
:10621B009000147403F022EF6423600302638F1267
:10622B007CEB900018E06439707CA3E064397076E5
:10623B00A3E064397070D23D900017E0FFB43108D1
:10624B00E490004AF00262E1EFB43208E490004BB4
:10625B00F00262F9EFB433028043900017E0FFB411
:10626B003408E490004CF0026327EFB43508E49057
:10627B00004DF002633DEFB43608E490004EF0029F
:10628B006353EFB437028015900017E0FFB4380961
:10629B009000497401F0026388EFB4390B7BFF7AED
:1062AB001279A8026395C23D900017E0FFB4301637
:1062BB00A3E0B43011A3E0B4300CA3E0B4300790EA
:1062CB000014740AF022EFB43113900018E0B430CC
:1062DB000C12B5945007900014740FF02290001715
:1062EB00E0B43211A3E0B4300C12B5945007900017
:1062FB00147414F022900017E0B43311A3E0B430FF
:10630B000C12B59450079000147419F022900017DA
:10631B00E0B4340FA3E0B4300A12B66F90001474DB
:10632B001EF022900017E0B4350FA3E0B4300A1230
:10633B00B6849000147423F022900017E0B4360F4B
:10634B00A3E0B4300A12B6999000147428F022908E
:10635B000017E0B43716A3E0B43011A3E0B4300C4F
:10636B00A3E0B43007900014742DF022900017E0D6
:10637B00B43811A3E0B4300C12B59450079000144C
:10638B007437F0227BFF7A12799812ABA690001427
:03639B0074FAF0A1
:01639E0022DC
:10AEA30090004F740BF09000507407F0E490005C36
:10AEB300F0A3F090005E7402F0E490005FF0A3F062
:10AEC3007BFF7A11796812ABA612A5C67F1E127D8D
:08AED3001D9000147432F022FE
:10AFEC00129841D39000D1E094019000D0E09400ED
:10AFFC00400A12ABA090001474FAF0227E017F2953
:10B00C001254937E007FD91254BD900053E09000EF
:03B01C0014F0220B
:10AAE3007BFF7A11799812ABA67BFF7A11797812E2
:10AAF300A5CC7F0E127D1D900019E0FF127CEB9018
:10AB0300001AE0FF127CEB7F1A127D1D90004F7438
:0FAB130010F09000507404F09000147432F0228F
:108B2100303E079000147403F02290001BE064397A
:108B31007041A3E06439703BA3E064397035900063
:108B41004F7411F09000507407F07BFF7A1379C8CD
:108B510012ABA6D23D900049E075F099A42469FEBC
:108B6100E5F034FF90005CF0CE12A5B77F1E127DB8
:108B71001D804212A5C67F1E127D1D1298B6503C63
:108B810090004F7411F09000507407F0900049E08C
:108B910075F099A42469FEE5F034FF90005CF0A320
:108BA100CEF090005E7403F090004AE0FF90005F09
:108BB100E4F0A3EFF09000147432F02212ABA09015
:068BC100001474FAF0221A
:10B01F00129841D39000D1E094059000D0E09400B5
:10B02F00400A12ABA090001474FAF0227E027F2B1C
:10B03F001254937E017F3B1254BD900053E0900059
:03B04F0014F022D8
:10AB22007BFF7A11799812ABA67BFF7A1179881292
:10AB3200A5CC7F0E127D1D900019E0FF127CEB90D8
:10AB4200001AE0FF127CEB7F1A127D1D90004F74F9
:0FAB520015F09000507404F09000147432F0224B
:1089C900303E079000147403F02290001BE06439D4
:1089D9007042A3E06439703CA3E0643970369000BA
:1089E9004F7416F09000507407F07BFF7A1379C822
:1089F90012ABA6D23D900049E0FF7E007C017D507C
:108A0900127EBBEF24A6FFEE340A12A5B27F1E1216
:108A19007D1D804812A5C67F1E127D1D12975150DB
:108A29004290004F7416F09000507407F09000497E
:108A3900E0FF7E007C017D50127EBBEF24A6FFEE95
:108A4900340A90005CF0A3EFF090005E7403F0909C
:108A5900004BE0FF90005FE4F0A3EFF09000147486
:0D8A690032F02212ABA090001474FAF0223B
:10B05200129841D39000D1E094059000D0E0940082
:10B06200400A12ABA090001474FAF0227E037F51C2
:10B072001254937E027F611254BD900053E09000FF
:03B0820014F022A5
:10AB61007BFF7A11799812ABA67BFF7A1279781262
:10AB7100A5CC7F0E127D1D900019E0FF127CEB9099
:10AB8100001AE0FF127CEB7F1A127D1D90004F74BA
:0FAB91001AF09000507404F09000147432F02207
:10855800303E079000147403F02290001BE0643949
:108568007042A3E06439703CA3E06439703690002F
:108578004F741BF09000507407F07BFF7A1379C892
:1085880012ABA6D23D900049E0FF7E007C027DEE52
:10859800127EBBEF2448FFEE342312A5B27F1E12D1
:1085A8007D1D806512A5C67F1E127D1D129E4290FC
:1085B80000D2E0FEA3E0FFD39400EE94004051EF18
:1085C80094FBEE9400504990004F741BF0900050BB
:1085D8007407F0900049E0FF7E007C027DEE127E79
:1085E800BBEF2448FFEE342390005CF0A3EFF0903B
:1085F800005E7403F09000D3E024FFFE9000D2E008
:1086080034FF90005FF0A3CEF09000147432F02293
:0A86180012ABA090001474FAF022D7
:10B08500129841D39000D1E094039000D0E0940051
:10B09500400A12ABA090001474FAF0227E047F5788
:10B0A5001254937E037F871254BD900053E09000A5
:03B0B50014F02272
:10A3B70090004F741FF09000507407F090005C7489
:10A3C70060F0A374CEF0E490005EF090004CE0FFE4
:10A3D70090005FE4F0A3EFF07BFF7A1179A812AB4E
:10A3E700A612A5C67F0F127D1D900019E0FF127CF3
:10A3F700EB90001AE0FF127CEB7F1E127D1D900090
:05A40700147432F02284
:10B0B800129841D39000D1E094FF9000D0E094FF23
:10B0C800400A12ABA090001474FAF0227E047F9B11
:10B0D8001254937E047F7B1254BD900053E090007D
:03B0E80014F0223F
:10A40C0090004F7424F09000507407F090005C742E
:10A41C0060F0A374CEF0E490005EF090004DE0FF8D
:10A42C0090005FE4F0A3EFF07BFF7A1179B812ABE8
:10A43C00A612A5C67F0F127D1D900019E0FF127C9D
:10A44C00EB90001AE0FF127CEB7F1E127D1D90003A
:05A45C00147432F0222F
:10B0EB00129841D39000D1E094FF9000D0E094FFF0
:10B0FB00400A12ABA090001474FAF0227E057F1563
:10B10B001254937E047FF51254BD900053E09000CF
:03B11B0014F0220B
:10A4610090004F7429F09000507407F090005C74D4
:10A4710060F0A374CEF0E490005EF090004EE0FF37
:10A4810090005FE4F0A3EFF07BFF7A1179C812AB83
:10A49100A612A5C67F0D127D1D900019E0FF127C4A
:10A4A100EB90001AE0FF127CEB7F1E127D1D9000E5
:05A4B100147432F022DA
:10B11E00129841D39000D1E094FF9000D0E094FFBC
:10B12E00400A12ABA090001474FAF0227E057F8FB5
:10B13E001254937E057F6F1254BD900053E0900021
:03B14E0014F022D8
:10B2A7003038079000147401F02290004F742EF08C
:10B2B7009000507407F07BFF7A1179D812ABA61271
:0EB2C700A5C67F1E127D1D9000147432F02269
:10AE3100303E07900014742FF02290001EE0643819
:10AE41006005A3E0B4390A12ABA090001474FAF0C3
:10AE5100227BFF7A12798812ABA690001EE0540F74
:09AE6100F55A9000147430F0223F
:10A6EA0090001EE064386005A3E0B4390A12ABA0FA
:10A6FA0090001474FAF0227BFF7A1179E812ABA663
:10A70A0090001EE0540FF55AD202D20B9000F8E0E6
:10A71A00F534125D447BFF7A1279B812ABA6C202F5
:09A72A00C20B90001474FEF02231
:10A2590090001EE0540FF55A303602D200125D56B6
:10A2690090026C7414F0C26730361B202704E54253
:10A2790070F9125D4DC2007BFF7A1279B812ABA654
:10A2890090001474FEF030371F20250AE54260065D
:10A2990012B6D63067F3125D4D7BFF7A1279B81288
:08A2A900ABA690001474FEF056
:01A2B100228A
:10A1FF00303956900015E0FF900048F0C239127CBC
:10A20F00EB900048E0FF12B7605021900048E0FF4C
:10A21F00900050E02417F582E43400F583EFF090BE
:10A22F000050E004F0900014E004F022900048E0A9
:10A23F00B42A079000147403F0227BFF7A127998E6
:0AA24F0012ABA690001474FAF0227E
:109AEF0030396A900015E0FF900048F0C239127CBF
:109AFF00EB900048E0FFB42A0B90004FE090001469
:109B0F00F0D23E22EFB4230B90004FE0900014F000
:109B1F00C23E22900048E0FF12B7605021900048EB
:109B2F00E0FF900050E02417F582E43400F583EF56
:109B3F00F0900050E004F0900014E004F0227BFF5E
:0E9B4F007A12799812ABA690001474FAF022E4
:10A8940030393F900015E0FF900048F0127CEBC285
:10A8A40039900048E0FFB42A0B90004FE090001468
:10A8B400F0D23E22EFB4230B90004FE0900014F04E
:10A8C400C23E227BFF7A12799812ABA690001474D0
:03A8D400FAF02275
:10999E0090004F7438F09000507407F090005C7493
:1099AE0060F0A374CEF090005E7456F0303D15E476
:1099BE0090005FF0A3F07BFF7A1379D812ABA6125A
:1099CE00A5C68032900049E024FFFEE434FF9000EB
:1099DE005FF0A3CEF07BFF7A13795812ABA612A5D7
:1099EE00C67F0C127D1D900019E0FF127CEB9000DB
:1099FE001AE0FF127CEB7F1E127D1D900014743254
:029A0E00F02244
:10A08F00129841D39000D1E094469000D0E0940014
:10A09F00400A12ABA090001474FAF0227E0C7F18C5
:10A0AF00125493900057E0FF601175F010A424989C
:10A0BF00F9740535F0FA7BFF12ABA6900058E0FF5C
:10A0CF00601175F010A42498F9740535F0FA7BFF30
:0CA0DF0012A5CC900053E0900014F02279
:109FD400900056E0FF7003303E45127D1D12B4110F
:109FE40012758D900170EFF0900054E05F90017055
:109FF400F060047F3180027F30127CEB303E20C25F
:10A004003E900170E090003760057431F080037475
:10A0140030F09000477401F090001474F0F0229036
:0EA024000059E0FF127D1D900014E004F022B0
:10A85000303940900015E0FF900048F0C239127C7A
:10A86000EB900048E0FFB42A079000147403F02234
:10A8700012B760500F900048E0900021F090001453
:10A88000E004F0227BFF7A12799812ABA6900014B4
:04A8900074FAF02244
:10AF4B00303932900015E0FF900048F0C239BF2A2B
:10AF5B00079000147403F022900048E0B42307908C
:10AF6B000014E004F0227BFF7A12799812ABA690C2
:06AF7B00001474FAF0223C
:105EDE00203D03025F70900017E064386003025F9C
:105EEE007090005FF0A3F012B4119000D4EEF0A306
:105EFE00EFF012758D900170EFF09000517401F07B
:105F0E00900021E0B4311C900170E0FF900054E04D
:105F1E00FEEF4E900170F0FD9000D4E0FEA3E0FF86
:105F2E0012754C900021E0B43018900054E0F4FF4C
:105F3E00900170E05FF0FD9000D4E0FEA3E0FF1250
:105F4E00754C900060E004F0700690005FE004F085
:105F5E00C3900060E0941490005FE09400408802CB
:105F6E006065203D03026001900017E0643360031A
:105F7E0002600190005FF0A3F012B4119000D4EE15
:105F8E00F0A3EFF012758D900170EFF09000517448
:105F9E0001F0900021E0B4311C900170E0FF900000
:105FAE0054E0FEEF4E900170F0FD9000D4E0FEA3A1
:105FBE00E0FF12754C900021E0B43018900054E0D0
:105FCE00F4FF900170E05FF0FD9000D4E0FEA3E0DE
:105FDE00FF12754C900060E004F0700690005FE0D8
:105FEE0004F0C3900060E094FA90005FE0940040EB
:105FFE0088805D12B4119000D4EEF0A3EFF012750C
:10600E008D900170EFF09000517401F0900021E03E
:10601E00B4311E900170E0FF900054E0FEEF4E9000
:10602E000170F0FD9000D4E0FEA3E0FF12754C80ED
:10603E001F900021E0B4301F900054E0F4FF900157
:10604E0070E05FF0FD9000D4E0FEA3E0FF12754C0F
:10605E0090001474FEF0227BFF7A12799812ABA690
:07606E0090001474FAF02207
:1093DC00900056E0FF7003303E68127D1D12B411F0
:1093EC009000D4EEF0A3EFF0E4900170F0900054F4
:1093FC00E0FF900170E0C39F50349000D4E475F00E
:10940C0001127F22AFF0FE12758D900171E4F0A372
:10941C00EFF0E0FF900170E02437F582E43400F5C2
:10942C0083EFF0127CEB900170E004F080BF303ED3
:10943C0011C23E900054E0900047F090001474F07C
:10944C00F022900050740AF0900059E0FF127D1D3C
:07945C00900014E004F0226F
:1096D800303975900015E0FF900048F0C239127CCF
:1096E800EB900048E0FFB42A079000147403F022BE
:1096F800EFB42308900014E004F0803912B76050EA
:1097080038900048E0FF900050E0FE04F074172EF7
:10971800F582E43400F583EFF0900054E02409FF6B
:10972800E433FE900050E0D39FEE6480F874809894
:109738004016900014E004F0227BFF7A1279981208
:09974800ABA690001474FAF022A3
:10AD0B00303937900015E0FF900048F0C239127CC3
:10AD1B00EB900048E0FFB42A079000147403F02274
:10AD2B00EFB42307900014E004F0227BFF7A127932
:0BAD3B009812ABA690001474FAF022EE
:10820800303D7B900017E06433707390005FF0A3FB
:10821800F012B4119000D4EEF0A3EFF09000507477
:108228000AF0E4900170F0900054E0FF900170E0D3
:10823800C39F502B9000D4E475F001127F22AFF059
:10824800FE900050E0FD04F074172DF582E4340030
:10825800F583E0FD12754C900170E004F080C89041
:108268000060E004F0700690005FE004F0C3900046
:1082780060E094FA90005FE094004095804E12B45C
:10828800119000D4EEF0A3EFF0900050740AF0E4DF
:10829800900170F0900054E0FF900170E0C39F508F
:1082A8002B9000D4E475F001127F22AFF0FE90000D
:1082B80050E0FD04F074172DF582E43400F583E0F6
:1082C800FD12754C900170E004F080C87BFF7A12B3
:0C82D80079B812ABA690001474FEF022DE
:109A800030396B900015E0FF900048F0C239127C2D
:109A9000EB900048E0FFB42A079000147403F02212
:109AA00012B760501A900048E0FF900050E0FE04AA
:109AB000F074172EF582E43400F583EFF080107B0C
:109AC000FF7A12799812ABA690001474FAF02290E3
:109AD0000054E02409FFE433FE900050E0D39FEEF1
:0F9AE0006480F87480984006900014E004F0222F
:1086E300900056E0FF7006203E0302878E127D1D28
:1086F30012B4119000D4EEF0A3EFF012758D125363
:10870300E2900054E0B401109000CDE0FF127CEB46
:108713009000CDE0900037F0900054E0B402209038
:1087230000CCE0FF127CEB9000CDE0FF127CEB90DD
:1087330000CCE0900037F09000CDE0900038F0904E
:108743000054E0640370309000CBE0FF127CEB90A8
:1087530000CCE0FF127CEB9000CDE0FF127CEB90AD
:1087630000CBE0900037F09000CCE0900038F09020
:1087730000CDE0900039F0303E11C23E900054E04D
:10878300900047F090001474F0F022900059E0FF3D
:10879300127D1D900050740AF0900014E004F02242
:10667A0012543850030267D6125410900170EFF08A
:10668A0090005AE0FEEFC39E50030267D6A3E0FFD4
:10669A00900170E0D39F40030267D6303D419000DD
:1066AA0017E06431703990005FF0A3F012B41190D2
:1066BA0000D4EEF0A3EFF0900170E0FD12754C905B
:1066CA000060E004F0700690005FE004F0C3900000
:1066DA0060E0943390005FE0940040D00267C630D7
:1066EA003D41900017E06432703990005FF0A3F0EA
:1066FA0012B4119000D4EEF0A3EFF0900170E0FD17
:10670A0012754C900060E004F0700690005FE0049F
:10671A00F0C3900060E0947090005FE0940040D075
:10672A000267C6303D40900017E06433703890002D
:10673A005FF0A3F012B4119000D4EEF0A3EFF09042
:10674A000170E0FD12754C900060E004F070069054
:10675A00005FE004F0C3900060E094FA90005FE00C
:10676A00940040D08056303D40900017E064387065
:10677A003890005FF0A3F012B4119000D4EEF0A3A9
:10678A00EFF0900170E0FD12754C900060E004F0AB
:10679A00700690005FE004F0C3900060E0941490EB
:1067AA00005FE0940040D0801312B4119000D4EE40
:1067BA00F0A3EFF0900170E0FD12754C7BFF7A12A6
:1067CA0079B812ABA690001474FEF02212ABA09016
:0667DA00001474FAF02225
:106511001254385003026670125410900170EFF05B
:1065210090005AE0FEEFC39E400BA3E0FF90017084
:10653100E0D39F4009900170E06003026670303D36
:1065410041900017E06431703990005FF0A3F012C0
:10655100B4119000D4EEF0A3EFF0900170E0FD12C1
:10656100754C900060E004F0700690005FE004F06C
:10657100C3900060E0943390005FE0940040D0024B
:106581006660303D41900017E06432703990005FE1
:10659100F0A3F012B4119000D4EEF0A3EFF090014B
:1065A10070E0FD12754C900060E004F07006900000
:1065B1005FE004F0C3900060E0947090005FE094AD
:1065C1000040D0026660303D40900017E0643370B7
:1065D1003890005FF0A3F012B4119000D4EEF0A354
:1065E100EFF0900170E0FD12754C900060E004F056
:1065F100700690005FE004F0C3900060E094FA90B0
:10660100005FE0940040D08056303D40900017E09C
:106611006438703890005FF0A3F012B4119000D488
:10662100EEF0A3EFF0900170E0FD12754C90006068
:10663100E004F0700690005FE004F0C3900060E0B9
:10664100941490005FE0940040D0801312B4119034
:1066510000D4EEF0A3EFF0900170E0FD12754C7BD9
:10666100FF7A1279B812ABA690001474FEF02212D0
:09667100ABA090001474FAF022B1
:1092CA00900056E0FF7003303E6A127D1D12B41101
:1092DA009000D4EEF0A3EFF012758D900170EFF0CC
:1092EA00129463E4900170F0900170E0FFC394045B
:1092FA005030E0FE24CBF582E43400F583E0FD74BF
:10930A00372EF582E43400F583EDF074CB2FF58225
:10931A00E43400F583E0FF127CEB900170E004F086
:10932A0080C6303E0FC23E9000477403F09000148E
:10933A0074F0F022900059E0FF127D1D90005074E5
:09934A000AF0900014E004F02286
:106D6A007F0A127A01900170EFF07003026EA1306F
:106D7A003D42900017E06431703A90005FF0A3F052
:106D8A0012B4119000D4EEF0A3EFF0900170E01469
:106D9A00FD12754C900060E004F0700690005FE010
:106DAA0004F0C3900060E0943390005FE0940040E8
:106DBA00CF026E89303D42900017E06432703A90FB
:106DCA00005FF0A3F012B4119000D4EEF0A3EFF03C
:106DDA00900170E014FD12754C900060E004F070B0
:106DEA000690005FE004F0C3900060E094709000A9
:106DFA005FE0940040CF026E89303D41900017E079
:106E0A006433703990005FF0A3F012B4119000D48B
:106E1A00EEF0A3EFF0900170E014FD12754C9000B3
:106E2A0060E004F0700690005FE004F0C390006038
:106E3A00E094FA90005FE0940040CF8042303D43F6
:106E4A00900017E06438703B90005FF0A3F012B432
:106E5A00119000D4EEF0A3EFF0900170E014FD124F
:106E6A00754C900060E004F0700690005FE004F05A
:106E7A00C3900060E0941490005FE0940040CF7BE0
:106E8A00FF801C12B4119000D4EEF0A3EFF0900131
:106E9A0070E014FD12754C900170E07BFF600E7A71
:106EAA001279B812ABA690001474FEF0227A127905
:0B6EBA003812ABA690001474FAF0220E
:10891900900056E0FF7006203E030289B4127D1DC7
:1089290012B4119000D4EEF0A3EFF012758D12532A
:10893900E29000D4E475F001127F22AFF0FE1275C7
:108949008D1253C69000CCE0FF900037F0A3F012CF
:108959007CEB9000CDE0FF127CEB9000D4E475F045
:1089690001127F22AFF0FE12758D1253C69000CB13
:10897900E0FF900039F09000CCE090003AF09000D0
:10898900CDE090003BF0127CEB9000CCE0FF127C34
:10899900EB9000CDE0FF127CEB303E0FC23E900021
:1089A900477405F090001474F0F022900059E0FF2C
:1089B900127D1D900050740AF0900014E004F0221A
:10607500900021E0540F75F00AA4FFA3E0540F2F00
:10608500900170F0FD900024E0540F75F00AA4FB18
:10609500AAF0900023E0540F75F064A42BFFE5F0FF
:1060A5003AFE900025E0540F7A002FFFEA3E90015A
:1060B50074F0A3EFF0EDC394014022900170E0D39A
:1060C50094145019900174E0FEA3E0FFC39401EE0F
:1060D50094004009D3EF94FAEE9400400A12ABA065
:1060E50090001474FAF022303D5E900017E06431A0
:1060F500705690005FF0A3F012B4119000D4EEF04A
:10610500A3EFF09000D4E475F001127F22AFF0FE0A
:10611500900170E0FD12754C9000D4E0FEA3E0FF05
:10612500900175E0FD12754C900060E004F070067A
:1061350090005FE004F0C3900060E0943390005F4E
:10614500E0940040B30261FB303D5D900017E064D0
:1061550032705590005FF0A3F012B4119000D4EEA8
:10616500F0A3EFF09000D4E475F001127F22AFF0B8
:10617500FE900170E0FD12754C9000D4E0FEA3E0A6
:10618500FF900175E0FD12754C900060E004F07021
:106195000690005FE004F0C3900060E0947090000A
:1061A5005FE0940040B3804E12B4119000D4EEF03D
:1061B500A3EFF09000D4E475F001127F22AFF0FE5A
:1061C500900170E0FD12754C900024E0540F75F0BD
:1061D5000AA4FF900023E0540F75F064A42FFF90EC
:1061E5000025E0540F2F900170F0FD9000D4E0FEE3
:1061F500A3E0FF12754C7BFF7A1279B812ABA6901B
:06620500001474FEF022FB
:10639F007F0D127A01EF701A900024E0B43010A331
:1063AF00E0B4300BA3E0B43006A3E0643060030226
:1063BF0064A9900028E0FF64306004EFB4350E90BC
:1063CF000029E0540FD3940540030264A9900028DC
:1063DF00E0FF64316004EFB4361190002DE0B4207B
:1063EF000790002CE0B420030264A9900028E0FF7E
:1063FF0064326004EFB4371190002CE0B4200790A2
:10640F00002BE0B420030264A9900028E0FF64335E
:10641F006004EFB43809900029E0B42002807B902B
:10642F000028E0FF64346005EF643970779000292D
:10643F00E0540F75F00AA4FFA3E0540F2F900170E2
:10644F00F0FD90002CE0540F75F00AA4FBAAF09019
:10645F00002BE0540F75F064A42BFFE5F03AFE908B
:10646F00002DE0540F7A002FFFEA3E900174F0A345
:10647F00EFF0EDC394014022900170E0D3941450DB
:10648F0019900174E0FEA3E0FFC39401EE94004065
:10649F0009D3EF94FAEE9400400A12ABA0900014C7
:1064AF0074FAF02212B4119000D4EEF0A3EFF09032
:1064BF000050740AF0E4900170F0900054E0FF90E7
:1064CF000170E0C39F502B9000D4E475F001127F50
:1064DF0022AFF0FE900050E0FD04F074172DF5820E
:1064EF00E43400F583E0FD12754C900170E004F088
:1064FF0080C87BFF7A1279B812ABA690001474FE95
:02650F00F02278
:108ED500900056E0FF7003303E73127D1D12B411F1
:108EE5009000D4EEF0A3EFF0E4900170F090005400
:108EF500E0FF900170E0C39F503F9000D4E475F00F
:108F050001127F22AFF0FE12758D900171E4F0A37E
:108F1500EFF0E0FF900170E02437F582E43400F5CE
:108F250083EFF0900171E0FEA3E0FF12758D127CD6
:108F3500EB900170E004F080B4303E11C23E900029
:108F450054E0900047F090001474F0F0229000591E
:108F5500E0FF127D1D900050740AF0D23C90001481
:048F6500E004F02212
:109D0800303965900015E0FF900048F0C239BF2A4D
:109D1800079000147403F022900048E0FFB4230871
:109D2800900014E004F0803DEF547FFF127CEB902C
:109D38000048E0547FFF900050E0FE04F074172EB6
:109D4800F582E43400F583EFF0900054E02409FF35
:109D5800E433FE900050E0D39FEE6480F87480985E
:099D68004006900014E004F02212
:10A6040030394B900015E0FF900048F0C239BF2A62
:10A61400079000147403F022900048E0FFB4230B69
:10A62400900014E004F0E004F0801012B760500FC2
:10A63400900048E0900052F0900014E004F0227B77
:0FA64400FF7A12799812ABA690001474FAF022E4
:108C6D00203903028D09900015E0FF900048F0C2F5
:108C7D0039BF2A079000147403F022900048E0FFDA
:108C8D00B4230A900014E004F0E004F02212B7605F
:108C9D00505B900052E0540F75F00AA4FF9000480D
:108CAD00E0540F2FF0E090110493FF900048F01264
:108CBD007CEB900048E0FF900050E0FE04F074174C
:108CCD002EF582E43400F583EFF0900054E0240992
:108CDD00FFE433FE900050E0D39FEE6480F8748083
:108CED0098900014E0400304F02214F0227BFF7AE8
:0D8CFD0012799812ABA690001474FAF022C0
:108DA500900056E0FF7003303E7A127D1D12B4111B
:108DB5009000D4EEF0A3EFF012758DC0079000D5AA
:108DC500E02401FF9000D4E03400FE12758DAD075C
:108DD500D0071254F5900061EEF0A3EFF012A65300
:108DE5009000CBE0FF127CEB9000CCE0FF127CEB17
:108DF5009000CDE0FF127CEB9000CBE0900037F0C7
:108E05009000CCE0900038F09000CDE0900039F073
:108E1500303E11C23E900054E0900047F09000149F
:108E250074F0F022900059E0FF127D1D90005074FF
:098E35000AF0900014E004F022A0
:109A100012B1B7900171EEF0A3EFF0D394E7EE949A
:109A2000035053D25012B4119000D4EEF0A3EFF0D3
:109A3000900171E0FEA3E0FF1254F4AD079000D452
:109A4000E0FEA3E0FF12754C900171E0FEA3E0FF81
:109A50001254F0AD079000D5E02401FF9000D4E04F
:109A60003400FE12754C7BFF7A1279B812ABA690C7
:109A7000001474FEF02212ABA090001474FAF022CD
:10B2D50030360B900120E0900006F012531B3038F9
:10B2E50005E4900006F030370E9000063034057402
:0EB2F5000AF080037428F0900014E004F022A8
:1083B800900006E060030284891277B330383E20CB
:1083C80059FD900264747EF0D2592059FD900264E0
:1083D8007450F0D2592059FD9000D6E075F00A8407
:1083E8004430900264F0D2592059FD9000D6E075CF
:1083F800F00A84E5F04430900264F0D259900053BA
:10840800E0127F3884316484366E8436788436820C
:1084180084368C843896843DA08442AA8447B484E8
:108428004CBE8436C80000845412B4B4801E80192F
:1084380012AC1B801712AC578012120078800D12F4
:108448000079800812AA23800312A55F30360F90A6
:10845800010CE0900001F0900014E004F0223038A4
:108468001A2059FD900264740DF0D2592059FD90DC
:108478000264740AF0D259C238C2359000147401EB
:02848800F022E0
:10B72000900001E070091253219000147401F0227E
:109C9E00303611900120E0900006F012531B900018
:109CAE0006E070FA30370C9000067405F09000064E
:109CBE00E070FAE4900170F030370C12B7DB1253FB
:109CCE00B612B8051253B630360C12B7E61253B6AA
:109CDE0012B8051253B6900170E004F0E0C394057B
:109CEE0040D630360E90010CE0900001F09000014D
:0A9CFE00E070FA9000147401F022E7
:0100120022CB
:01006A002273
:010076002267
:108E3E003038079000147402F02230370A203407BD
:108E4E009000147401F022303611900120E0900051
:108E5E0006F012531B900006E070FA30370C9000AB
:108E6E00067405F0900006E070FA3036209000F59A
:108E7E00E0F53612B7E6E4900170F01253B69001A9
:108E8E0070E004F0E0C3940A40F112B805303720C8
:108E9E009000F6E0F53612B7DBE4900170F0125355
:108EAE00B6900170E004F0E0C3940A40F112B805E8
:108EBE0030360E90010CE0900001F0900001E07051
:078ECE00FAE4900014F02209
:010077002266
:10B1E90030272C203929900013741EF0787EE6FF51
:10B1F900547FFE900EFB93900015F0303C0DEF301C
:10B20900E709EE900F0B93900015F0D239C227226F
:10B2190030252C203929900013741EF0787CE6FF24
:10B22900547FFE900EFB93900015F0303C0DEF30EB
:10B23900E709EE900F0B93900015F0D239C2252241
:105BA800900274E0FF65797003025D4330390302A7
:105BB8005D43900013741EF0EFD394FA4005E4900F
:105BC8000274F0900274E0FF04F074752FF582E41B
:105BD8003402F583E0FF647F7003025D43D239BF6E
:105BE8005D07900015745DF022BF5B079000157487
:105BF8005BF022BF30079000157430F022BF3107E8
:105C08009000157431F022BF32079000157432F0FD
:105C180022BF33079000157433F022BF3407900079
:105C2800157434F022BF35079000157435F022BF83
:105C380036079000157436F022BF370790001574A8
:105C480037F022BF38079000157438F022BF3907A3
:105C58009000157439F022BF23079000157423F0C3
:105C680022BF2A07900015742AF022BF410790002E
:105C7800157441F022BF42079000157442F022BF0C
:105C880043079000157443F022BF64079000157411
:105C980044F022203C03C23922BF610790001574EA
:105CA80061F022BF62079000157462F022BF63079B
:105CB8009000157463F022BF64079000157464F0B7
:105CC80022BF65079000157465F022BF6607900033
:105CD800157466F022BF67079000157467F022BF3D
:105CE80068079000157468F022BF69079000157462
:105CF80069F022BF6A07900015746AF022BF6B072B
:105D0800900015746BF022BF6C07900015746CF04E
:105D180022BF6D07900015746DF022BF6E079000CA
:105D280015746EF022BF6F07900015746FF022BFD4
:0B5D380070079000157470F022C23953
:015D4300223D
:10002E00E4900170F0900170E0FFC39420501574BD
:10003E00172FF582E43400F5837420F0900170E000
:05004E0004F080E12236
:0FB76000EFC394304007EFD39439500122C32236
:10984100900020E0FD6420602E90001FE0540F7511
:10985100F00AA4FBAAF090001EE0540F75F064A476
:109861002BFFE5F03AFEED540F7C002FFFEC3E900C
:1098710000D0F0A3EF803190001FE0FD6420900044
:109881001E601AE0540F75F00AA4FFED540F7C001E
:109891002FFEEC35F09000D0F0A3CE800BE0540FFA
:1098A100FF9000D0E4F0A3EFF0E024FFF09000D0AF
:0598B100E034FFF0228D
:109E420090001DE0FD6420602B90001CE0540F7513
:109E5200F00AA4FBAAF090001BE0540F75F064A472
:109E62002BFFE5F03AFEED540F7C002FFFEC3E9005
:109E720000D2802E90001CE0FD642090001B601A2E
:109E8200E0540F75F00AA4FFED540F7C002FFEEC96
:109E920035F09000D2F0A3CEF022E0540FFF9000F4
:079EA200D2E4F0A3EFF0226F
:10B59400900019E0540F75F00AA4FFA3E0540F2F94
:10B5A400900049F0D394004006E09415500122C362
:01B5B4002274
:1098B600E4900170F0900170E0FFC394335064EFC0
:1098C60075F003A4241BF582E4340FF583E493FFBB
:1098D60090001BE0FEEF6E7042900170E0FF75F0A5
:1098E60003A4241CF582E4340FF583E493FE900070
:1098F6001CE0FDEEB50524EF75F003A4241DF582EA
:10990600E4340FF583E493FF90001DE0FEEFB50607
:109916000A900170E090004AF0D322900170E004B2
:05992600F08092C32255
:10975100E4900170F0900170E0FFC3947050677560
:10976100F003EFA424B4F582E5F0340FF583E4931C
:10977100FF90001BE0FEEF6E7044900170E0FF75FA
:10978100F003A424B5F582E5F0340FF583E493FEEC
:1097910090001CE0FDEEB5052575F003EFA424B69D
:1097A100F582E5F0340FF583E493FF90001DE0FEB0
:1097B100EFB5060A900170E090004BF0D3229001C2
:0897C10070E004F0808FC32268
:107A010074172FF582E43400F583E0FE64316003DE
:107A1100027A95900170F0900170E0FDC3943350AB
:107A21007074182FF582E43400F583E0FCED75F0F5
:107A310003A4241BF582E4340FF583E4936C7049AD
:107A410074192FF582E43400F583E0FD900170E0B4
:107A5100FC75F003A4241CF582E4340FF583E49350
:107A6100B50526741A2FF582E43400F583E0FDECA8
:107A710075F003A4241DF582E4340FF583E493B576
:107A81000507900170E004FF22900170E004F0808E
:107A9100867F0022EE64326003027B22900170F047
:107AA100900170E0FEC39470507474182FF582E455
:107AB1003400F583E0FD75F003EEA424B4F582E50E
:107AC100F0340FF583E4936D704C74192FF582E453
:107AD1003400F583E0FE900170E0FD75F003A4240D
:107AE100B5F582E5F0340FF583E493B50628741AF1
:107AF1002FF582E43400F583E0FE75F003EDA42454
:107B0100B6F582E5F0340FF583E493B506089001EC
:107B110070E02434FF22900170E004F080827F0045
:047B2100227F00229D
:10946300EFC394339000CB50397431F0EF75F003B0
:10947300A4241BF582E4340FF583E4939000CCF02D
:10948300EF75F003A4241CF582E4340FF583E49311
:109493009000CDF0EF75F003A4241DF582E4340FA2
:1094A300803A7432F075F003EFA4241BF582E5F0E3
:1094B300340FF583E4939000CCF075F003EFA4240C
:1094C3001CF582E5F0340FF583E4939000CDF0753D
:1094D300F003EFA4241DF582E5F0340FF583E49344
:0594E3009000CEF02214
:10B66F00900019E0540F75F00AA4FFA3E0540F2FB8
:05B67F0090004CF022D8
:10B68400900019E0540F75F00AA4FFA3E0540F2FA3
:05B6940090004DF022C2
:10B69900900019E0540F75F00AA4FFA3E0540F2F8E
:05B6A90090004EF022AC
:10B4110090005EE0FF7E0090005FE0FCA3E0FD1283
:10B421007EBB90005DE02FFF90005CE03EFE90004F
:0AB4310055E07C002FFFEC3EFE22E8
:10B4B400303608900037E0FF1200863037089000DD
:10B4C40037E0FF12005E30380D2059FD900037E060
:07B4D400900264F0D259223E
:10A55F00E4900170F0900047E0FF900170E0FEC3BF
:10A56F009F503F74372EF582E43400F583E0FF905F
:10A57F000171E4F0A3EFF0303605E0FF12008630F2
:10A58F003708900172E0FF12005E30380D2059FD40
:10A59F00900172E0900264F0D259900170E004F0E3
:03A5AF0080B32254
:10AC1B00303838E4900170F0900170E0FFC3940479
:10AC2B00502974CB2FF582E43400F583E0FF9001BB
:10AC3B0071E4F0A3EFF02059FD900172E0900264F3
:0CAC4B00F0D259900170E004F080CD229E
:10AC5700303838E4900170F0900170E0FFC394053C
:10AC6700502974CB2FF582E43400F583E0FF90017F
:10AC770071E4F0A3EFF02059FD900172E0900264B7
:0CAC8700F0D259900170E004F080CD2262
:010078002265
:010079002264
:10AA230030383CE4900170F0900054E0FF900170E6
:10AA3300E0FEC39F502974372EF582E43400F5837A
:10AA4300E0FF900171E4F0A3EFF02059FD90017253
:10AA5300E0900264F0D259900170E004F080C922C2
:0C005E0012B6411253B612B80C0253B691
:0C00860012B6581253B612B80C0253B652
:1077B300E4900170F0900171F0A3F0900173F090E8
:1077C30000D1E02401FD9000D0E03400FCC3ED942F
:1077D3000AEC94005007A3E004900173F0D3ED94F6
:1077E30063EC9400405D9000D1E02401FB9000D055
:1077F300E03400FA7C007D64AF03FE127ECD90017D
:1078030070EFF0E075F064A4FFC3EB9FFFEA95F01F
:10781300FE7C007D0A127ECD900171EEF0A3EFF0A5
:107823009000D1E004FF900170E075F064A4FEC302
:10783300EF9EFF900172E075F00AA4FEC3EF9E90E5
:107843000173F09000D1E02401FF9000D0E03400F8
:10785300FED3EF9409EE940040207C007D0A127E53
:10786300CD900171EEF0A3EFF0E075F00AA4FF9064
:1078730000D1E004C39F900173F0900170E02430C5
:10788300F0900172E02430F0900171E03400F09048
:107893000173E02430F030361D900170E0FF1200D8
:1078A30086900172E0FF120086900173E0FF1200E0
:1078B300867F2A12008630371D900170E0FF120088
:1078C3005E900172E0FF12005E900173E0FF120010
:0778D3005E7F2A12005E2215
:06ABA0007BFF7A12790828
:10ABA6008B188A19891A20382E7F01127D1DE49090
:10ABB6000170F0900170E0FFC39410501AAB18AA10
:10ABC60019A91A8F82758300127E7CFF127CEB9086
:08ABD6000170E004F080DC22B4
:10A5B20090005CF0EFA3F090005E7403F0E4900072
:0AA5C2005FF0A3F07BFF7A127958D6
:10A5CC008B178A18891920382E7F11127D1DE49063
:10A5DC000170F0900170E0FFC39410501AAB17AAF1
:10A5EC0018A9198F82758300127E7CFF127CEB9068
:08A5FC000170E004F080DC2294
:10B43B007BFF7A1279C812A5CCE4900170F09001D1
:10B44B0070E0FF7E00900E9793FD12754C9001708B
:0AB45B00E004F0E0C3940240E52293
:109353007BFF7A1279D812A5CCE4900173F0E490E4
:109363000171F0A3F0E4900170F0900173E075F0E7
:1093730099A42402FBE435F0FA900171E0FEA3E026
:10938300FF7C007D03127EBBEF2BFFEE3AFE9001C4
:1093930070E0FD7A002FFFEA3EFEED900E9993FDFB
:1093A30012754C900170E004F0E0C3940340BB904D
:1093B3000172E004F07006900171E004F0C39001C3
:1093C30072E09433900171E094004099900173E04E
:0993D30004F0E0C394144086226A
:109121007BFF7A1279E812A5CCE4900173F0E49008
:109131000171F0A3F0E4900170F0900173E0FF7E03
:10914100007C017D50127EBBEF24F6FBEE340BFA5E
:10915100900171E0FEA3E0FF1C7D03127EBBEF2BAB
:10916100FFEE3AFE900170E0FD7A002FFFEA3EFE2D
:10917100ED900E9C93FD12754C900170E004F0E0AF
:10918100C3940340B5900172E004F0700690017140
:10919100E004F0C3900172E09470900171E09400DA
:0F91A1004093900173E004F0E0C39414408022E7
:109B5D007BFF7A1279F812A5CCE4900174F0A3F092
:109B6D00E4900170F0900170E0FBC39403502E90CF
:109B7D000174E0FEA3E0FF7C007D03127EBBEF24A9
:109B8D0036FFEE3426FEEB2FFFEC3EFEEB900E9FE4
:109B9D0093FD12754C900170E004F080C890017532
:109BAD00E004F07006900174E004F0C3900175E0DC
:0B9BBD009488900174E0941340A622ED
:01007A002263
:01007E00225F
:01007F00225E
:109BC8007BFF7A13793812A5CCE4900171F0A3F0E9
:109BD800E4900170F0900170E0FBC39456502E9011
:109BE8000171E0FEA3E0FF7C007D56127EBBEF24EE
:109BF800CEFFEE3460FEEB2FFFEC3EFEEB900EA5A1
:109C080093FD12754C900170E004F080C8900172C9
:109C1800E004F07006900171E004F0C3900172E076
:0B9C28009414900171E0940040A6220B
:10B4DB007BFF7A13794812ABA612B43B129353122B
:10B4EB009121129B5D12007A12007E12007F129B3B
:07B4FB00C8127D3A027D4CEE
:10B46500E49000D4F0A3F0FFFE12758D9000A8EFD4
:10B47500F09000D5E02401FF9000D4E03400FE12E6
:08B48500758D9000D6EFF02256
:108A7600756D01756E00756FE9E4900378F0A3F0EB
:108A8600900378E0FAA3E0FBC39456EA94005040C2
:108A96009000A8E075F056A42478FFE5F03460CF86
:108AA6002BCF3AFE9000D4F0A3EFF012758DAB6D8C
:108AB600056FE56FAA6E7002056E14F9EF127EA9B6
:108AC600900379E004F070B8900378E004F080B089
:108AD600900116E024FF924B900115E024FF92329C
:108AE600900135E0F537900136E0F53890011CE04D
:108AF60024FF924A90011BE024FF923390011AE072
:108B06007004D2558002C255900113E024FF9223CF
:0A8B16009000A974FFF09000AAF08F
:018B20002232
:10A0EB00756D01756E01756F48E4900378F0A3F000
:10A0FB00900378E0FEA3E0FFC39414EE9400503B72
:10A10B007C007D56127EBBEF24F9FFEE3460FE908F
:10A11B0000D4F0A3EFF012758DAB6D056FE56FAA50
:10A12B006E7002056E14F9EF127EA9900379E004AC
:0BA13B00F070BD900378E004F080B5E8
:01A1460022F6
:10A14700756D01756E01756F5CE4900378F0A3F08F
:10A15700900378E0FEA3E0FFC39414EE9400503B15
:10A167007C007D56127EBBEF24FEFFEE3460FE902E
:10A1770000D4F0A3EFF012758DAB6D056FE56FAAF4
:10A187006E7002056E14F9EF127EA9900379E00450
:0BA19700F070BD900378E004F080B58C
:01A1A200229A
:1091B0008F17E4900170F0900170E0FBC3940350AE
:1091C0003E9000A8E075F099A42469FDE5F034FF15
:1091D000FCE51775F003A42DFFE5F03CFEEB7C00E9
:1091E0002FFFEC3EFE12758D900170E024DEF582BB
:1091F000E43400F583EFF0900170E004F080B89063
:1092000000DEE0FE54019000D7F0EE54029000D84A
:10921000F09000DEE054049000D9F0EE5408900085
:10922000DAF09000DEE054109000DBF09000DFE018
:0D9230009000DCF09000E0E09000DDF02206
:108FFD008F17E4900170F0900170E0FBC394035063
:10900D00449000A8E0FF7E007C017D50127EBBEFF6
:10901D0024A6FDEE340AFCE51775F003A42DFFE53B
:10902D00F03CFEEB7C002FFFEC3EFE12758D9001A7
:10903D0070E024DEF582E43400F583EFF0900170EA
:10904D00E004F080B29000DEE0FE54019000D7F015
:10905D00EE54029000D8F09000DEE054049000D958
:10906D00F0EE54089000DAF09000DEE0541090001D
:10907D00DBF09000DFE09000DCF09000E0E090008D
:03908D00DDF022F1
:068BC7008F178C188D19B8
:108BCD00E4900378F0A3F0E51924FFFFE51834FFD6
:108BDD00FE7C007D03127EBBAA06AB07AE17E51720
:108BED0025E0CE75F0EEA4FFE5F02EFEEF2448FF54
:108BFD00EE3423CF2BCF3AFE900379E02FFF900375
:108C0D0078E03EFE12758D900379E024DEF582E466
:108C1D003400F583EFF0900379E004F070069003D3
:108C2D0078E004F0C3900379E09403900378E09426
:108C3D000040949000DEE0FE54019000E4F0EE540C
:108C4D00029000E5F09000DEE054049000E6F09014
:0F8C5D0000DFE09000E7F09000E0E09000E8F02A
:018C6C0022E5
:103CE2007BFF7A0079A612ABA612ADF7E490025FD1
:103CF200F0A3F090017304F0900173E0C3941540B7
:103D020003023EB9900174E4F0A304F0C39001757C
:103D1200E094FB900174E094004003023EB09001F5
:103D220073E0FF7E007C027DEE127EBBEF2448FF33
:103D3200EE342390005CF0FAA3EFF0FB900175E003
:103D420024FFFF900174E034FFFE7C007D03127EAD
:103D5200BBEF2BFFEE3AFE12758DEF54029000DEA0
:103D6200F0900175E024FFFF900174E034FFFE7CC7
:103D7200007D03127EBB90005DE02FFF90005CE0AF
:103D82003EFE12758DEF54049000E1F09000DEE0EB
:103D92007003023E9C9000E1E07003023E9C9001A1
:103DA20074E0FEA3E0FF7C007D03127EBB90005D09
:103DB200E02FFF90005CE03ECF24FECF34FFFE12E6
:103DC200758D9000DFEFF0900174E0FEA3E0FF7CC0
:103DD200007D03127EBB90005DE02FFF90005CE04F
:103DE2003ECF24FFCF34FFFE12758D9000E0EFF03E
:103DF200FD9000DFE0FF1254F5900171EEF0A3EFA9
:103E0200F04E7003023E9C90025FE475F001127F57
:103E120022AFF0FE900173E0FD12A73390025FE43F
:103E220075F001127F22AFF0FE900175E0FD12A73E
:103E32003390025FE475F001127F22AFF0FE900032
:103E4200DFE0FD12A73390025FE475F001127F22DA
:103E5200AFF0FE9000E0E0FD12A733D3900260E0E5
:103E6200948890025FE0941340307BFF7A0079B728
:103E720012ABA690025FE0FEA3E07802CEC313CE9F
:103E820013D8F9F0EE90025FF09000057414F090F0
:103E92000005E0700302416A80F5900175E004F0CC
:103EA2006003023D0E900174E004F0023D0E9001A9
:103EB20073E004F0023CFAE4900170F0900170E0CB
:103EC200FBC394334003023FF19000A8E075F099E0
:103ED200A42469FDE5F034FFFCEB75F003A42DFF8B
:103EE200E5F03CFE90005CF0A3EFF012758D9000BF
:103EF200DEEFF054049000E1F09000DEE054109008
:103F020000E2F09000E1E07003023FE8A3E07003FA
:103F1200023FE890005DE02401FF90005CE0340085
:103F2200FE12758D9000DFEFF090005DE02402FF3D
:103F320090005CE03400FE12758D9000E0EFF0FD21
:103F42009000DFE0FF1254F5900171EEF0A3EFF064
:103F52004E7003023FE890025FE475F001127F2287
:103F6200AFF0FE7D1512A73390025FE475F00112E7
:103F72007F22AFF0FE900170E0FD12A73390025F46
:103F8200E475F001127F22AFF0FE9000DFE0FD1237
:103F9200A73390025FE475F001127F22AFF0FE902A
:103FA20000E0E0FD12A733D3900260E09488900213
:103FB2005FE0941340307BFF7A0079B712ABA69092
:103FC200025FE0FEA3E07802CEC313CE13D8F9F06D
:103FD200EE90025FF09000057414F0900005E0701E
:103FE2000302416A80F5900170E004F0023EBEE4F3
:103FF200900170F0900170E0FBC3947040030241A5
:104002004B9000A8E0FE75F050A4FFE5F02EFEEF05
:1040120024A6FDEE340AFCEB75F003A42DFFE5F0B7
:104022003CFE90005CF0A3EFF012758DEF5404900B
:1040320000DEF090005CE0FEA3E0FF12758DEF540D
:10404200109000E1F09000DEE07003024142900027
:10405200E1E0700302414290005DE02401FF900024
:104062005CE03400FE12758D9000DFEFF090005D91
:10407200E02402FF90005CE03400FE12758D900097
:10408200E0EFF0FD9000DFE0FF1254F5900171EED9
:10409200F0A3EFF09000DEE070030241429000E1F5
:1040A200E07003024142900171E07002A3E07003EC
:1040B20002414290025FE475F001127F22AFF0FEEE
:1040C2007D1612A73390025FE475F001127F22AFD2
:1040D200F0FE900170E0FD12A73390025FE475F0EC
:1040E20001127F22AFF0FE9000DFE0FD12A73390B5
:1040F200025FE475F001127F22AFF0FE9000E0E073
:10410200FD12A733D3900260E0948890025FE0949E
:1041120013402D7BFF7A0079B712ABA690025FE0C5
:10412200FEA3E07802CEC313CE13D8F9F0EE9002CC
:104132005FF09000057414F0900005E0602A80F8AA
:10414200900170E004F0023FF690025FE0FEA3E00F
:104152007802CEC313CE13D8F9F0EE90025FF07B53
:09416200FF7A0079C812ABA62215
:10A65300AB07AA067C007D64127ECDEF44309000E8
:10A66300CBF07C007D64AF03AE02127ECD7E007F13
:10A673000ACFCDCFCECCCE127ECDEF4430A3F0AEF9
:10A6830002AF037C007D64127ECD7E007F0ACFCDB6
:0DA69300CFCECCCE127ECDED4430A3F02210
:10B1B700900022E0540F75F00AA4FDACF090002136
:10B1C700E0540F75F064A42DFFE5F03CFE900023DA
:10B1D700E0540F7C002FFFEC3EFE900171F0A3EFCF
:02B1E700F02254
:10A50B002A2A3132333435362A2A2A2A3132333445
:10A51B0035302A2A44313233343536373839302AFC
:10A52B002341424320464C45582049562020412088
:10A53B00332E30302020202020534C4156452020F4
:10A54B002020202020202020204D415354455220F4
:04A55B00202020207C
:10886300303F23C23F787EE6540F90A51F939001BB
:108873008AF09000077432F09000EAE0601612ADBF
:108883008112A7C3800E900007E07008900176F074
:10889300900187F0304049C240787CE6540F90A5A0
:1088A3001F93900189F09000087432F090025EE00B
:1088B300FF60069000E9E07009EF70099000EBE0BB
:1088C300600312A77C90025EE0FF60069000E9E07F
:1088D3007003EF700312AD4620341312B151800EB2
:1088E300900008E07008900177F0900186F0900204
:1088F30074E0FF657960149000ECE06018EFD394A6
:10890300FA4005E4900274F0027F5E900009E07083
:0689130004900273F02243
:10AD4600900177E0FF04F0EF90A50B93FF90018947
:10AD5600E0FEEF6E6011EEB42A089001777401F000
:10AD66008005E4900177F0900177E0B40A0C125365
:0BAD760021E4900177F0D237D2412297
:10AD8100900176E0FF04F0EF90A50B93FF90018A0C
:10AD9100E0FEEF6E6011EEB42A089001767401F0C6
:10ADA1008005E4900176F0900176E0B40A0C12532C
:0BADB10021E4900176F0D236D241225E
:10A77C00900186E0FF04F0747D2FF582E43401F53E
:10A78C0083E0FF900189E0FEEF6E6011EEB42308C8
:10A79C009001867401F08005E4900186F0900186AA
:10A7AC00E0B4091212532D125321120056E49001F9
:07A7BC0086F0D237D23522EE
:10A7C300900187E0FF04F0747D2FF582E43401F5F6
:10A7D30083E0FF90018AE0FEEF6E6011EEB4230880
:10A7E3009001877401F08005E4900187F090018760
:10A7F300E0B4091212532D125321120056E49001B2
:07A8030087F0D236D23522A6
:10B15100900179E0FF04F0EF90A51593FF9001892C
:10B16100E0FEEF6E6011EEB42A089001797401F0EF
:10B171008005E4900179F0900179E0B40A04E4F0EB
:03B18100D2422295
:10B35F0090017D7423F0A3F0E4FF74ED2FF582E4E8
:10B36F003400F583E0FE747F2FF582E43401F5831A
:0CB37F00EEF00FBF06E49001857423F08F
:01B38B00229F
:109F7300127C48127D3A127D4C7F01127D1D7BFFBE
:109F83007AA5792F12ABA690011AE07BFF60067ABF
:109F9300A5793F80047AA5794F12A5CC900005746A
:109FA3001EF0E490017BF090017CF0FF74AB2FF581
:109FB30082E43400F583E4F074BB2FF582E43400CB
:109FC300F583E4F00FBF10E4900005E070FA027D22
:019FD3003A53
:10965E0090017BE0FFD3940F501FEF04FF127D1D8E
:10966E00900189E0FF90017BE0FE04F074AB2EF5D3
:10967E0082E43400F583EF804C7F01127D1DE4906F
:10968E000170F0900170E0FFC3940F5030E0FE24A3
:10969E00ACF582E43400F583E0FD74AB2EF582E484
:1096AE003400F583EDF074AB2FF582E43400F583CE
:1096BE00E0FF127CEB900170E004F080C69001890F
:0A96CE00E0FF9000BAF0127CEB22DE
:1095680090017CE0FFD3940F5020EF2411FF127D6F
:109578001D90018AE0FF90017CE0FE04F074BB2E90
:10958800F582E43400F583EF804C7F11127D1DE4F1
:10959800900170F0900170E0FFC3940F5030E0FE2E
:1095A80024BCF582E43400F583E0FD74BB2EF5821B
:1095B800E43400F583EDF074BB2FF582E43400F554
:1095C80083E0FF127CEB900170E004F080C690010C
:0B95D8008AE0FF9000CAF0127CEB223A
:107F5E00900273E0FF702C900274E0FE04F07475D2
:107F6E002EF582E43402F583E090017AF090000958
:107F7E007432F090017AE0FEB41B02D241EEB47E70
:107F8E00028064EFB4012A900274E0FF04F074756D
:107F9E002FF582E43402F583E090017AF090000927
:107FAE007432F090017AE0B45002803BE490027398
:107FBE00F0900273E06402703A900274E0FF04F0F5
:107FCE0074752FF582E43402F583E090017AF09017
:107FDE0000097432F09000D6E075F00A844430FF48
:107FEE0090017AE0B50707900273E004F022E49066
:107FFE000273F0900273E064037044900274E0FF29
:10800E0004F074752FF582E43402F583E090017A62
:10801E00F09000097432F0E4900273F09000D6E014
:10802E0075F00A84E5F04430FF90017AE0B5070F51
:10803E00E4900014F0D238D235D239C250C2512257
:105D4400755900125D5F50FB22755900125DE850D1
:105D5400FB22755900125D9F50FB22758400E559A2
:105D640075F003A4905D6C73025E04025E13025E20
:105D740031025E1A025E3D025E44025E4C025E1314
:105D8400025E5A025E1A025E6A025E73025E0402D8
:105D94005E13025E81025E1A025E8D758400E5590F
:105DA40075F003A4905DAC73025E04025E13025EA0
:105DB40031025E1A025E3D025E44025E04025E131C
:105DC400025E31025E1A025E3D025E44025E3D02E4
:105DD4005E44025E4C025E13025E8F025E1A025E35
:105DE4006A025E8D758400E55975F003A4905DF533
:105DF40073025E04025E13025E81025E1A025E8D0D
:105E0400C2FA125E9F125E9F759B000559C3223031
:105E1400F9020559C32230F912E59A20E7FB125E14
:105E24009FD2FA125E9F125E9F0559C322C2FA12D4
:105E34005E9F759B040559C32275411E0559C322F3
:105E4400E54170020559C322C2FA125E9F125EC078
:105E5400F59B0559C322C2FA125E9F125ECF440716
:105E6400F59B0559C322125EB1F5420559C322754B
:105E7400840F30DE04E54270020559C322C2FA12CF
:105E84005E9F759B080559C322D322C2FA125E9FF6
:095E9400125ECF4405F59B05598F
:105E9D00C322000000000000000000000000000010
:105EAD0000000022905EB8E55A93225A5A5A5A5A67
:105EBD00FAFAFA905EC7E55A932200B45AE12D879B
:105ECD007ADB905ED6E55A93220000000000008038
:015EDD008044
:101EE700C0D0C000C001C083C082C0E0C0F0C0073E
:101EF700A292304B01B3787BE233F208E233F20867
:101F0700E233F208E233F208E233F208E233F2088E
:101F1700E233F208E233F208E233F208E233F2087E
:101F2700E233F208E233F208E233F208E233F2086E
:101F3700E233F208E233F208E233F208E233F2085E
:101F4700E233F208E233F208E233F208E233F2084E
:101F5700E233F208E233F208E233F208E233F2083E
:101F6700E233F208E233F208E233F208E233F2082E
:101F7700E233F208E233F208E233F208E233F2081E
:011F8700E277
:101F880033F208E233F208E233F208E233F208E20D
:101F980033F208E233F2305C3278A2E218202303ED
:101FA80030E728E21820E723E21830E71EE218207D
:101FB800E719E21830E714E21830E70FE21820E7D3
:101FC8000AE21820E705E21830E70302212B7550D2
:101FD80000E2183392435003755038752300E21815
:101FE80033921C500363501CE21833921B50036356
:101FF800500EE21833921A5003635046E218339297
:10200800195003635023E218339218852351500363
:10201800635051752300E21833921C5003635068D3
:10202800E21833921B5003635075E21833921A502A
:102038000363507AE218339219500363503DE21853
:10204800339218852352500363501F752300E218FA
:1020580033921F500363504FE21833921E500363AC
:102068005026E21833921D5003635052E2183392FF
:072078001C5003635029E234
:10207F001833921B5003635015E21833921A500312
:10208F0063500BE2183392195003635045E2183333
:10209F0092188523535003635062E21833921C50F9
:1020AF0003635031E21833921B5003635019E21847
:1020BF0033921A500363500DE21833921950036391
:1020CF005007E21833921885235450036350437519
:1020DF002300E21833921EE21833921DE218339256
:1020EF001CE21833921BE21833921AE2183392193A
:1020FF00E218339218852355E5556550701EA2439B
:10210F0092449000A3E551F09000A4E552F09000A6
:10211F00A5E553F09000A6E554F0D24612213FD02A
:10212F0007D0F0D0E0D082D083D001D000D0D02221
:10213F00C0D0C000C0E0302D4EE562B40833A230ED
:10214F00B392B37880E66036167885E6A2E7303230
:10215F0001B3923092B2A2E77881E633F67882E645
:0C216F0033F67883E633F67884E633F626
:10217B007885E633F6D56203756208D0E0D000D0DF
:10218B00D022C254D0E0D000D0D022D0E0D000D0AA
:10219B00D022C0D0C000C001C083C082C0E0C0F05C
:1021AB00A292204A01B37863E213F208E213F20819
:1021BB00E213F208E213F208E213F208E213F20858
:1021CB00E213F208E213F208E213F208E213F20848
:1021DB00E213F208E213F208E213F208E213F20838
:1021EB00E213F208E213F208E213F208E213F20828
:1021FB00E213F208E213F208E213F208E213F20818
:10220B00E213F29023517863E20893139217E208DA
:10221B0093139216E20893139215E20893139214F8
:08222B00E20893139213E2088C
:1022330093139212E20893139211E20893139210EC
:10224300852256E20893139217E20893139216E23B
:102253000893139215E20893139214E208931392CE
:1022630013E20893139212E20893139211E2089374
:10227300139210852257E20893139217E2089313DF
:102283009216E20893139215E20893139214E2084C
:1022930093139213E20893139212E2089313921189
:1022A300C210852258305C3DE5569026A185572201
:1022B300301602058393602D14F875F003A490255E
:1022C300522582F582E5F03583F583E493F9A3E49F
:1022D30093902451655893C965579329B4010050CD
:1022E300048844D22F1222FAD0F0D0E0D082D083D7
:1022F300D001D000D0D022302B26788616E670206D
:1023030076087889E6A2E1303301B392B292B3A2A0
:01231300E1E8
:102314007887E613F67888E613F67889E613F622CA
:10232400EF90255175F003A42582F582E58335F0FD
:10233400F583C22B7400937887F67401937888F63A
:102344007402937889F6C22DC22CD22B220000008D
:102354000000000000000000000000000000000079
:102364000000000000000000000000000100000068
:102374000000000000000000000000000100000058
:102384000000000001000000010001010100000044
:102394000000000000000000000000000100000038
:1023A4000000000001000000010001010100000024
:1023B4000000000001000000010001010100000014
:1023C40001000101010001010101010101000000FE
:1023D40000000000000000000000000001000000F8
:1023E40000000000010000000100010101000000E4
:1023F40000000000010000000100010101000000D4
:1024040001000101010001010101010101000000BD
:1024140000000000010000000100010101000000B3
:10242400010001010100010101010101010000009D
:10243400010001010100010101010101010001018B
:102444000101010101010101010101010100010179
:102454000201020203010202030203030401020255
:10246400030203030402030303030304050102023A
:102474000302030304020303040304040502030325
:10248400040304040503040404040505060102020C
:102494000302030304020303030304040502030306
:1024A40004030304050304040504050506020303E9
:1024B40004030404050304040504050506030404D5
:1024C40005040505060405050605060607010202BE
:1024D40003020303040203030403040405020303C5
:1024E40004030404050304040504050506020303A8
:1024F4000403040405030404050405050603040495
:10250400050405050604050506050606070203037A
:102514000403040405030404050405050603040474
:102524000504050506040505060506060703040457
:102534000504050506040505060506060704050544
:1025440006050606070506060706070708FDD00C5C
:1025540073700E3CF01AAF101E7F9022EC7026D6DA
:10256400F02ACBB02CA3F032BEB03417D03CB6D096
:10257400461FB04E77F050F950526AB056DE90586C
:10258400BA306ACF3072D270745CD076E8F0786B6F
:10259400D098E5709AF8309CBB50A40F70AA7A705A
:1025A400B26730B45DB0B8FCB0C26F50C655D0CA83
:1025B4003D90D489B0DA94F0DCD790E463B0EA0BB0
:1025C400F0F43170F8DD310AB571148FF118D1D1FE
:1025D40026EB512AF6112C8B71463F5148B1F14A32
:1025E400ACB14CC4F152D9B1546D915A2EF162BDC3
:1025F400116687916A9AD16CF29172D5517819F16A
:102604008C71B192D8D19A32D1AA47D1B25A91B42D
:1026140052F1C67531CC1D71D2A951DCD0B1E85E3E
:1026240011EA2B11F2EED212F392147D3216973284
:1026340026D8B232C5F234F7124AEA524C9F5254A9
:10264400A5D2582B725A7552644FD268C1726ADC93
:10265400326C78D2865F128C83729C4EB2A66972F9
:10266400AC1C72B433D2CC18F2EABB330CCE3314A4
:102674001EB32803F32EE51332F8533498735848E5
:0D268400F36472736845738617B394731383
:10269100A63C93B221D3B41B53B829B3C641F3D896
:1026A1000000000000000000000000000000000029
:1026B100000000000000006A000000000000620D40
:1026C1000000000000000000006F00480000000052
:1026D1000000000000000000000000006C2200006B
:1026E10000000000000000000000000000005B008E
:1026F100000000000000000000004100001E4759DA
:10270100000000260000001D000010000035000040
:10271100003D006B0043000000000000004B00057D
:10272100000000000000003800230000000000004D
:10273100000000000000004C00000000000000004C
:102741000000000000000000000000003200000452
:1027510000000000000000000000126000370A00C5
:1027610000000000000000000000000800006113EC
:1027710046000000000000254D34000057291100DB
:1027810000000000006400000000000000000000E4
:1027910000003A4A00002E4F190000001F000000FF
:1027A1000000006300000000000000270000001B83
:1027B100000000000000000B5F3C006E5D44000063
:1027C100006D000000000000000000530000360012
:1027D10000283F5E00000000000000000300003000
:1027E1000070000000690040670000000000005513
:1027F1000000420000210000000000001500000060
:102801000000000000000000005C00170000002034
:10281100000068020054000E58001C000000000077
:102821000000005A000000000000002F0000002BF3
:102831000000000024000000660039000000005183
:1028410000000009005200000045000000000000E7
:1028510000310000002A0C000000001A00000000F6
:1028610000560000334E0000000000000000000090
:10287100002C1400003B07003E0000000000000097
:1028810000000000001800001600502D060049004D
:102891000000000000000000650F000000010000C2
:1028A100000000000000060000000600060005020E
:1028B10006000600060004040600050402080600DE
:1028C10000000600060006000600040806000600D7
:1028D10006000508060006000210060006000301B6
:1028E1000000060006000202060006000440060081
:1028F1000600041006000600060006000600060099
:102901000600051006000600060006000600060087
:10291100010106000600060006000302060006008B
:10292100000006000600050106000402020406007C
:1029310006000600060006000600060006000480E8
:10294100060002010420060006000600060006003B
:102951000600060006000600060006000600060046
:102961000600060004010600060006000600060037
:102971000310060006000600060006000600060019
:102981000600060006000600060003080600060011
:102991000600060003040600060006000600060005
:10489100758400C2CA85CC4885CD4775CC0075CDDD
:1048A10000D2CA10CF02D25B32305B0BC25BE5474C
:1048B100C3943640028001227891798F7B06E7F616
:1048C1001819DBFAA64718A648AA48AB47AE02AFAB
:1048D10003EEC4035407FEEFC403FF54F84EFEEF8A
:1048E1005407FF7803798CC3E79AFC09E79BFD091C
:1048F10050066304FF6305FFC3EC9EED9F5074D81F
:10490100E6789979977C06E7F61819DCFAA6031878
:10491100A6027994AE02AF03EEC423541FFEEFC486
:1049210023FF54E04EFEEF541FFF7803C3E79AFCC8
:1049310009E79BFD0950066304FF6305FFC3EC9E75
:10494100ED9F502FD8E678927A007B007C007904A5
:10495100EA26FA08EB36FB08EC3400FCD9F2EC133A
:0D496100FCEB13FBEA13FAEC13EB13F54625
:10496E00EA13F545D22122302131C2211249AA5033
:10497E002A854C4D854B4C854A4B85494A850749BE
:10498E00302013E54F6F600EE507B54A0EB54B0BA1
:10499E00B54C08B54D0585074ED22222904AC5E585
:1049AE004693FF9049F123232582F582E583340057
:1049BE00F5831249D0400A0F1249D040040F124914
:1049CE00D022E493F9A3E493FAA3E493FBA3E49334
:1049DE00FCA3C3E5459AE546995007C3EC9545EB14
:1049EE00954622EA25DD89DD89D324D324CBD2CB8B
:1049FE00D2C4DBC4DBBE39BE39B7CAB7CAB18EB1B9
:104A0E008EAB87AB87A59CA59CA000A0009A969A1A
:104A1E009695D895D891E591E58D858D8588AF8849
:104A2E00AF840C840C7F9A7F9A7B497B49771B77E6
:104A3E001B730F730F6F276F276B576B5767AB6720
:104A4E00AB642C642C60C660C65D795D795AFE5AE3
:104A5E00FE5970597057E257E25661566154E75449
:104A6E00E7537453745207520750A050A04F404F53
:104A7E00404DE64DE64C934C934B414B4149F54925
:104A8E00F548B548B547764776463E463E45084515
:104A9E0008432A432A40E440E43F533F533E3E3E00
:104AAE003E3C943C943A863A8639183918380500BB
:104ABE000000000000000032323232323232323226
:104ACE0032323232323232323232323232323232B8
:104ADE0032323232323232323232323232323232A8
:104AEE003232323232323232323232323232323298
:104AFE00313130302F2E2D2D2D2C2C2B2A292928DB
:104B0E0027262525242323222120201F1E1E1D1C7F
:104B1E001C1B1A1A1A1A19191918181817171717F9
:104B2E00161616161515151514141414131313132F
:104B3E00121212121111111110101010100F0F0F5E
:104B4E000F0F0E0E0E0E0D0D0D0D0C0C0C0C0B0B87
:104B5E000B0B0B0B0A0A0A0A0A09090909090908AB
:104B6E0008080808080707070707070606060606C7
:104B7E0006060505050505050404040404040403DE
:104B8E0003030303030302020202020202010101F4
:104B9E0001010101010101010101010000000000FC
:104BAE0000000000000000000000000000000000F7
:104BBE0000000000000000302C0D852F8A852E8C01
:0A4BCE00D28CB2B1D2A932C28C22FF
:10701D00C007C0007F01127D1D7F4C127CEB7F5499
:10702D00127CEB7F52127CEB7F20127CEB2045040F
:10703D007F3080027F31127CEB7F20127CEB90023F
:10704D0032E0785D125489785D8607430730127CF3
:10705D00EB088607430730127CEB750720127CEB9B
:10706D00900233E0785D125481785D8607430730D6
:10707D00127CEB088607430730127CEB088607432A
:10708D000730127CEB750720127CEB900234E07810
:10709D005D125489785D8607430730127CEB0886B4
:1070AD0007430730127CEB750720127CEBD000D024
:1070BD000722C007C0007F11127D1D7F4C127CEB93
:1070CD00750720127CEB2049047F3080027F31123E
:1070DD007CEB7F20127CEB9001F9E0785D125489F6
:1070ED00785D8607430730127CEB0886074307302F
:1070FD00127CEB750720127CEB9001FAE0785D12A3
:10710D005481785D8607430730127CEB0886074370
:10711D000730127CEB088607430730127CEB7507AE
:10712D0020127CEB9001FBE0785D125489785D862E
:10713D0007430730127CEB088607430730127CEBC0
:10714D00750720127CEB9001FCE0785D1254897874
:10715D005D8607430730127CEB0886074307301224
:07716D007CEBD000D00722EB
:106AA800003800512372461765340E5F2D7C481953
:106AB8006B3A1C4D3F6E5A0B7928124331605405CE
:106AC8007726001F3D227A654758756A48570F1088
:106AD800322D6877554A120D2F301D02203F6778F6
:106AE8005A45006245270B694E2C157750321E7C9B
:106AF8005B39294B6C0E224067053C5E791B375584
:106B0800721052301775593B1C7E472502604C2E77
:106B1800096B7B193E5C701235576E0C2B49650763
:106B28002042264463012D4F680A33517614385A9F
:106B38007D1F0F6D4A28046641231A785F3D117343
:106B48005436741631537F1D3A58610324466A0837
:106B58002F4D5D3F187A56341371482A0D6F432123
:106B680006644F2D0A68442601635A381F7D513345
:106B78001476660423416D0F284A73113654781A27
:106B88003D5F1D7F583A16745331086A4D2F0361D3
:106B98004624345671133F5D7A18214364062A4807
:106BA8006F0D690B2C4E620027457C1E395B7715EB
:106BB8003250402205674B290E6C553710725E3CE7
:106BC8001B793B597E1C305275172E4C6B09254793
:106BD800600212705735197B5C3E076542200C6EC7
:106BE800492B004307440D4E0A49195A1E5D145794
:106BF8001350317236753C7F3B78286B2F6C2566B5
:026C0800226107
:108D0A00788576ACA249E433FFC4333354C0FE906D
:108D1A0001FBE0FD541F25E04EFE9001F9E0FC54F2
:108D2A0010C4540F4E7884F6EC540FC454F0FE90DD
:108D3A0001FAE0FC54F0C4540F4E7883F6EC540F59
:108D4A00C454F0FE9001FCE0FC541EC3134E78821A
:108D5A00F6EF3395E0FE74A82FF582746A3EF58328
:108D6A00E493FFED906AAA93FEEF6EFF9001F9E09B
:108D7A00906ACA936FFF9001FAE0906AEA936FFFD4
:108D8A00EC906BEA936F7881F69001FCE030E00496
:0B8D9A00E64480F6D254788076282250
:10A4B600758401309914C299204C0F9001F7E07011
:10A4C60009D24CD29C789A7604223098379001F8BB
:10A4D600E06401702DE55B75F00584205211248D32
:10A4E600F582E43401F583E599F0C298D25222242C
:10A4F600A2F582E43401F583E599F0C298C252D2FE
:05A506005322C298225F
:1082E4007584012098030283AA204E13209A0DE579
:1082F400997009D24ED24F755C0AF55BC2982290F0
:1083040001F8E0FF6401702CE55B75F005842052F0
:1083140010248DF582E43401F583E599F0D252807E
:108324001024A2F582E43401F583E599F0C252D217
:1083340053C29822EFB4021AAB6D056FE56FAA6EB3
:108344007002056E14F9E599127EA99001F8740380
:1083540080209001F8E0FFB4031CAB6D056FE56F5E
:10836400AA6E7002056E14F9E599127EA99001F8BF
:108374007404F0C29822EFB4042990022AE0FF04A6
:10838400F074012FF582E43402F583E599F0C29884
:1083940090022AE0B4281C90022C7401F0E49001AD
:1083A400F8F022C2982230990AC2999001F7E0703D
:0483B40002C252228D
:10B50200204D2212534643E740755C0AE4F55B90F6
:10B5120001F7F09001F8F0C24CD24D758401759894
:06B5220090C29CF5992285
:109F100090022BE0705C90036FE0FF7025D39001FE
:109F2000FEE094869001FDE094674008E4F0A3749D
:109F300002F0800E9001FEE02428F09001FDE03454
:109F400000F09001FEE02FFF9001FDE03400FE12D2
:109F5000758D90036FE02401F582E43402F583EF00
:109F6000F090036FE004F0E0B42807E4F090022BD7
:039F700004F022D8
:1090900090022CE070030291209001FFE0FEA3E01B
:1090A000FFC39402EE94005006E490022CF022904C
:1090B000036FE07C002FFFEC3EFE12758D90036F76
:1090C000E02401F582E43402F583E0FD6F6017903F
:1090D000036FE0FF900200E02FFF9001FFE03400FB
:1090E000FE12754CD25090036FE004F0E0642870DB
:1090F0002F90022CF090036FF09001FFE0FEA3E0B0
:10910000FFBE2008BFD205E490036FF0EF64024E6B
:10911000700E30500BC250128A7612A0EB12A1478B
:01912000222C
:109DDA00304C6475840190023EE0B40D00505590F9
:109DEA009DF0F8282873029E17029E1A029E1D02F1
:109DFA009E20029E23029E26029E29029E2C029EDD
:109E0A002F029E32029E35029E38029E3B02B30307
:109E1A0002B6AE02A8D702AC9302B57102001E02C6
:109E2A00B18402AFB702ACCF02A91A02B60F02B3CD
:089E3A00B902B5F412B62922A9
:10B30300789AE67028759898755C0AF55B9000A8A2
:10B31300E0B4010790023E7404F022E49001F8F0D7
:0EB323009001F7F090023EE004F01253432236
:10B6AE009001F87401F0E49001F7F0C25290023E5E
:04B6BE00E004F02292
:10A8D7009000A8E01475F005A4B55B19E4B5F01570
:10A8E700759898125346E49001F7F09001F8F090AC
:10A8F700023E7404F0E55B75F00584AFF0BF01120A
:10A90700C253E49001F7F09001F804F090023EE0A2
:03A9170004F02227
:10AC9300E55B75F00584AFF0BF043020531EE55B20
:10ACA30075F00584FF248DF582E43401F583E4F027
:10ACB30074A22FF582E43401F583E4F0E49001F704
:0CACC300F09001F8F090023EE014F02246
:10B571009000A8E075F005A424FDB55B159000A925
:10B58100E0F599E49001F7F09001F8F090023EE0C7
:03B5910004F022A1
:0D001E009000AAE0F59990023EE004F02267
:10B184009000A8E0FD75F005A4FFE55BB50723E496
:10B19400B5F01FEDB4140790023E7409F022125367
:10B1A40043E49001F7F0C2529001F8F090023EE0BF
:03B1B40004F02282
:10AFB700E55BB46412125346E49001F7F09001F890
:10AFC700F090023E7409F0E55B75F00584AFF0BFC1
:10AFD7000112C253E49001F7F09001F804F09002D7
:05AFE7003EE004F02231
:10ACCF00E55B75F00584AFF0BF043020531EE55BE4
:10ACDF0075F00584FF248DF582E43401F583E4F0EB
:10ACEF0074A22FF582E43401F583E4F0E49001F7C8
:0CACFF00F09001F8F090023EE014F0220A
:10A91A00E55B6465703C90022BE0B4012F756D0114
:10A92A00756E01756FFDE49001F7F09001F8F0750E
:10A93A008401AB6D056FE56FAA6E7002056E14F99E
:10A94A00127E63F59990023EE004F02290023E7472
:03A95A000CF022DC
:10B60F00758401AB6DAA6EA96F127E63F599E490F4
:0AB61F000229F090023EE004F02240
:10B3B900758401900229E0FF04F074012FF582E4FD
:10B3C9003402F583E0F599900229E0D39428400BE3
:0CB3D900E490022BF090023EE004F02211
:10B5F400E55BB46915C24CC24DE490018BF0900137
:0BB60400F7F09001F8F090023EF022F9
:10B62900C24CC24DE4F55B90018BF09001F7F090AC
:08B6390001F8F090023EF0223E
:10A36100304E5275840190023FE0B40A0050439090
:10A37100A377F828287302A39502A39802A39B024E
:10A38100A39E02A3A102A3A402A3A702A3AA02A3BC
:10A39100AD02A3B002AF8102AE6A02AEDB02B5D557
:10A3A10002B73002B3E502A9E202AF1302B5B5026A
:06A3B100B70F12B74022B5
:10AF8100E55B70317598989000A8E0B401131253F5
:10AF910046E49001F8F09001F7F090023F7403F05D
:10AFA10022125343C252E49001F8F09001F7F0905D
:06AFB100023FE004F02263
:10AE6A009000A8E01475F005A4B55B11E4B5F00DE7
:10AE7A0075989812534690023F7403F022E55B7569
:10AE8A00F00584AFF0BF0110C253C2529001F874AA
:09AE9A0001F090023FE004F022F7
:10AEDB00E55B75F00584AFF0BF042C20531EE55BDA
:10AEEB0075F00584FF248DF582E43401F583E4F0DD
:10AEFB0074A22FF582E43401F583E4F0E49001F8B9
:08AF0B00F090023FE014F02277
:10B5D5009000A8E075F005A424FDB55B1175840104
:0FB5E5009000A9E0F599C25290023FE004F022D5
:10B730007584019000AAE0F59990023FE004F022A0
:10B3E5009000A8E0FFB4140790023F7406F022EF26
:10B3F50075F005A4B55B14E4B5F010125343900243
:0CB405003FE004F0C252E49001F8F02295
:10A9E200E55B75F00584AFF0BF0111C253C252900E
:10A9F20001F87401F090023FE004F022E55BB464D8
:10AA02001F12534390022CE0700B9001F8F0900259
:10AA12003F7408F022E49001F8F090023F7409F0CC
:01AA22002211
:10AF1300E55B75F00584AFF0BF042C20531EE55BA1
:10AF230075F00584FF248DF582E43401F583E4F0A4
:10AF330074A22FF582E43401F583E4F0E49001F880
:08AF4300F090023FE014F0223F
:10B5B500E55BB4651A756D01756E01756FFFE490F5
:10B5C500022AF090023F7409F09001F87402F0220B
:10B70F00E55BB4690BC24EE49001F8F090023FF094
:01B71F002207
:10B74000C24EE49001F8F09001F7F090023FF02231
:10740C00789DE660011678A3E6600116900000E016
:10741C00600214F0900002E0600214F0900001E0B1
:10742C00600214F0900003E0600214F0900004E09D
:10743C00600214F0900010E0600214F090000FE075
:10744C00600214F0900253E0600214F090025CE0D1
:10745C00600214F0789F16E6600302754B789F76F5
:10746C000A789EE6600116E542600215429000051E
:10747C00E0600214F0900006E0600214F090000747
:10748C00E0600214F0900008E0600214F090000933
:10749C00E0600214F090000AE0600214F090000B1F
:1074AC00E0600214F090000DE0600214F090000E09
:1074BC00E0600214F0900256E0600214F078A4E64A
:1074CC0060011690026CE0600214F090026FE060B4
:1074DC000214F0900270E0600214F078A016E670CE
:1074EC005E78A0760A900012E0600214F078A6E6AE
:1074FC001846600708E6161870011690025DE060E9
:10750C000214F090025EE0600214F090026AE060F7
:10751C000214F0900272E0600214F078A116E6708A
:10752C001E78A1760A900013E0600214F078A2167F
:10753C00E6700C78A27606900011E0600214F0223E
:10804E00535155452020434F53202053454E534501
:10805E00004F4E20202020202020202020202020D5
:10806E0020004F46462020202020202020202020A7
:10807E0020200024242424242424242424242424DE
:10808E0024242424242424242424242424242424A2
:10809E002424242424242424242424242424242492
:1080AE00242424231A1B1C1D1E1F202122242424B9
:1080BE0024242424000102030405060708090A0BE0
:1080CE000C0D0E0F10111213141516171819242457
:1080DE0024242424000102030405060708090A0BC0
:1080EE000C0D0E0F10111213141516171819242437
:1080FE0024242400000AAB0D55100012AB155518A0
:10810E00001AAB1D55200022AB255528002AAB2D99
:0D811E0055300032AA355538003AAA3D55BB
:10B52800751F01E51FC394155018AF1F74B62FF58A
:10B5380082E43401F583E0FFEF60037F0122051FF9
:04B5480080E17F001F
:01B54C0022DC
:10A2B200205455128622EF6401704D900119E0FF7F
:10A2C200EF24FF92499001F6E0FF74E02FF582E45B
:10A2D2003401F583E0FF9001F9EFF09001F6E0FF21
:10A2E20074CB2FF582E43401F583E0FF9001FAEF9D
:10A2F200F09001F6E0FF9001FBEFF01256B49001EE
:09A30200FCEFF0128D0AD22D22AD
:10862200900171E4F0A3E4F0900174E4F0A3E4F0AB
:10863200900170E4F0900170E0FFEFC394154003E5
:108642000286C69001F6E0FFEFD394144006900133
:10865200F67401F09001F6E0FF74B62FF582E4346F
:1086620001F583E0FF900173EFF0900173E0FFEFFB
:10867200B401159001F6E0FF74B62FF582E43401DF
:10868200F5837402F07F0122900173E0FFEFB402E0
:1086920024900171E0FEA3E0FFEF4E70189001718B
:1086A200E4F0A37401F09001F6E0FF7E0090017403
:1086B200EEF0A3EFF09001F6E004F0900170E00418
:1086C200F0028637900171E0FEA3E0FFEF4E7004E6
:1086D2007F002222900175E0FF9001F6EFF07F010A
:0186E2002275
:10848A00900171E4F0A3E4F0900174E4F0A3E4F045
:10849A00900170E4F0900170E0FFEFC3941540037F
:1084AA0002853B9001F6E0FFEFD394144006900159
:1084BA00F67401F09001F6E0FF74B62FF582E43409
:1084CA0001F583E0FF900173EFF0900173E0FFEF95
:1084DA0060509000A8E0FF9001F6E0FEEE6F604267
:1084EA00900173E0FFEFB401159001F6E0FF74B656
:1084FA002FF582E43401F5837402F07F01229001A2
:10850A0071E0FEA3E0FFEF4E70189001F6E0FF7EE7
:10851A0000900174EEF0A3EFF0900171E4F0A374FF
:10852A0001F09001F6E004F0900170E004F002849A
:10853A009F900171E0FEA3E0FFEF4E70047F0022DE
:0E854A0022900175E0FF9001F6EFF07F012214
:1056B4009000A8E0FFEFD3941440037F20229003CE
:1056C40073E4F0900372E4F09000A8E0FF9003709C
:1056D400EFF0900114E0FFEFD3940650030257A8B3
:1056E400900371E4F0900371E0FFEFC3941540035D
:1056F4000257A1900370E0FFEFB415069003707495
:1057040001F0900370E0FF748C2FF582E43401F50E
:1057140083E0FFEF64FF7076900370E0FF74472F1F
:10572400F582E43401F583E0FF9000A8E0FE7447BD
:105734002EF582E43401F583E0FEEEC39F404F90E2
:1057440000A8E0FF900370E0FEEEB507069003703A
:10575400E0FF22900370E0FF74472FF582E43401E8
:10576400F583E0FF900372E0FEEFD39E40209003A8
:1057740070E0FF900373EFF0900370E0FF74472F25
:10578400F582E43401F583E0FF900372EFF09003B7
:1057940071E004F0900370E004F00256E9900373A2
:1057A400E0FF2222900371E4F0900371E0FFEFC365
:1057B40094154003025864900370E0FFEF70069064
:1057C40003707414F0900370E0FF748C2FF582E47E
:1057D4003401F583E0FFEF64FF7076900370E0FF1F
:1057E40074472FF582E43401F583E0FF9000A8E0CC
:1057F400FE74472EF582E43401F583E0FEEEC39F88
:10580400404F9000A8E0FF900370E0FEEEB507065D
:10581400900370E0FF22900370E0FF74472FF5823D
:10582400E43401F583E0FF900372E0FEEFD39E4081
:1058340020900370E0FF900373EFF0900370E0FF9B
:1058440074472FF582E43401F583E0FF900372EF8F
:10585400F0900371E004F0900370E014F00257AD8F
:05586400900373E0FF5A
:01586900221C
:10586A009000A8E0FFEFD3941440037F2022900316
:10587A0077E4F0900376E4F0900114E0FFEFD3941C
:10588A0006500302594F9000A8E0FFEF04FF90036F
:10589A0074EFF0900375E4F0900375E0FFEFC394A2
:1058AA00154003025948900374E0FFEFD394144063
:1058BA00069003747401F0900374E0FF748C2FF562
:1058CA0082E43401F583E0FFEF64FF7062900374B1
:1058DA00E0FF74472FF582E43401F583E0FF90007E
:1058EA00A8E0FE74472EF582E43401F583E0FEEE6B
:1058FA00C39F403B900374E0FF74472FF582E43462
:10590A0001F583E0FF900376E0FEEFD39E402090FE
:10591A000374E0FF900377EFF0900374E0FF74479D
:10592A002FF582E43401F583E0FF900376EFF090DF
:10593A000375E004F0900374E004F00258A29003A7
:10594A0077E0FF22229000A8E0FFEF14FF90037493
:10595A00EFF0900375E4F0900375E0FFEFC3941540
:10596A004003025A04900374E0FFEF700690037438
:10597A007414F0900374E0FF748C2FF582E4340100
:10598A00F583E0FFEF64FF7062900374E0FF7447F1
:10599A002FF582E43401F583E0FF9000A8E0FE745D
:1059AA00472EF582E43401F583E0FEEEC39F403BC7
:1059BA00900374E0FF74472FF582E43401F583E025
:1059CA00FF900376E0FEEFD39E4020900374E0FF41
:1059DA00900377EFF0900374E0FF74472FF582E4A9
:1059EA003401F583E0FF900376EFF0900375E0044D
:0F59FA00F0900374E014F0025961900377E0FF1E
:015A0900227A
:10B6C2009000A8E0FFEFD3941440037F2022900063
:04B6D200A8E0FF22CB
:107685009001F5E0FFEFD3941440069001F57401E5
:10769500F0900170E4F09001F5E0FF74CB2FF582D6
:1076A500E43401F583E0FF9001F5E0FE74A12EF5C9
:1076B50082E43401F583E0FEEEB507269001F5E09E
:1076C500FF74E02FF582E43401F583E0FF9001F5C6
:1076D500E0FE748C2EF582E43401F583E0FEEE6F56
:1076E50060069001707401F09001F5E0FF748C2F35
:1076F500F582E43401F583E0FF9000A8E0FEEF6E2B
:10770500600E9000A8E0FF9001F5E0FEEE6F703A84
:10771500900170E0FFEF60439001F5E0FFEFD39437
:107725001550149001F5E0FF74B62FF582E434018D
:10773500F5837401F080249001F5E0FF74B62FF510
:1077450082E43401F583E4F080119001F5E0FF74E3
:10775500B62FF582E43401F583E4F0900170E0FF83
:10776500EF60449001F5E0FF74A12FF582E4340148
:10777500F583E0FF9001F5E0FE74CB2EF582E4344D
:1077850001F583EFF09001F5E0FF748C2FF582E4AD
:107795003401F583E0FF9001F5E0FE74E02EF582FB
:0E77A500E43401F583EFF09001F5E004F022EA
:106C0A00900239E0FFEF6003026CC590000BE0FFD1
:106C1A00EF70037F012212A9A0EFB40103120096BC
:106C2A0012A9A0EF70031200562046037F00221219
:106C3A00A9A0EF64016003026CC530467BC24620FE
:106C4A00360920370620380312701D9000A4E0FF91
:106C5A00900235EFF09000A5E0FF900236EFF09039
:106C6A0000A3E0FF900237EFF0900237E0FFEFB4A5
:106C7A001F14900233E0FF900236E0FEEEB50706DD
:106C8A001200567F0122900232E0FF900235E0FEA8
:106C9A00EEB5070E900233E0FF900236E0FEEE6F8B
:106CAA0060099002397401F07F002290010BE0FF25
:106CBA0090000BEFF07F00227F0022900239E0FF64
:106CCA00EF64016003026D6790000BE0FFEF700351
:106CDA007F012212A9A0EFB4010312009612A9A003
:106CEA00EF70031200562046037F0022C24612703C
:106CFA001D9000A4E0FF900235EFF09000A5E0FFA0
:106D0A00900236EFF09000A3E0FF900237EFF09088
:106D1A000237E0FFEFB41F14900233E0FF9002360F
:106D2A00E0FEEEB507061200567F0122900232E01D
:106D3A00FF900235E0FEEEB50720900233E0FF90A7
:106D4A000236E0FEEEB5071290010BE0FF90000B51
:106D5A00EFF0900239E4F07F00227F00227F0022C8
:10A9A000900102E0FFEF600D12534940047F0180E7
:10A9B000027F002222900103E0FFEF601390010468
:10A9C000E0FFE532D39F40047F0122227F00222254
:10A9D000900104E0FFE532C39F50047F0122227FF3
:02A9E000002253
:109D7100900170E4F0900170E0FFEFC3940A505835
:109D8100900170E0FF74262FF582E43401F583E041
:109D9100FFEFB42013900170E0FF743E2FF582E4D1
:109DA1003401F5837426F022900170E0FF74262FB0
:109DB100F582E43401F583E0FFEF90808193FF9019
:109DC1000170E0FE743E2EF582E43401F583EFF07C
:099DD100900170E004F0809D2275
:1067E00090023BE0FFEF600302689690000DE0FF2F
:1067F000EF70037F012212A9A0EFB40103120096EB
:1068000012A9A0EF700312005690023AE0FFEFB415
:1068100001062022037F002290023AE0FFEFB4023B
:1068200006202F037F002212A9A0EF64017064905C
:10683000023AE0FFEF6401702130221EC222E54FD0
:10684000654E600990023B7401F07F0022900110B8
:10685000E0FF90000DEFF07F002290023AE0FFEFA2
:106860006402702F302F2CC22F90023DE544F0902F
:10687000023DE0FF90023CE0FEEE6F600990023BBB
:106880007401F07F0022900110E0FF90000DEFF006
:106890007F00227F002290023BE0FFEF6401600353
:1068A00002694390000DE0FFEF70037F012212A9FF
:1068B000A0EFB4010312009612A9A0EF700312001A
:1068C0005690023AE0FFEFB401062022037F002237
:1068D00090023AE0FFEFB40206202F037F0022125D
:1068E000A9A0EF6401705A90023AE0FFEFB4011CD6
:1068F000302219C222E54FB54E1290023BE4F090CF
:106900000110E0FF90000DEFF07F002290023AE0CE
:10691000FFEF6402702B302F28C22F90023DE54418
:10692000F090023DE0FF90023CE0FEEEB5071290D1
:10693000023BE4F0900110E0FF90000DEFF07F00CB
:04694000227F002290
:10B249008F7A9000F5E0FF8F36AF7AEF3395E0FE05
:10B25900EF25E0FFEE33FE74012FF58274813EF590
:0FB2690083E493F508740193F509D229D20C22DE
:109EA9007BFF7A80794E12ABA6125349400B7BFF98
:109EB9007A80795F12A5CC80097BFF7A807970124C
:109EC900A5CC7F17127D1DAF321253E29000CBE073
:109ED900FF127CEB9000CCE0FF127CEB9000CDE010
:109EE900FF127CEB7F1C127D1DAF311253E29000F3
:109EF900CBE0FF127CEB9000CCE0FF127CEB9000F2
:079F0900CDE0FF127CEB220A
:0BB7C5007508027509ABD229D20C22D6
:0BB7D00075081A7509ABD229D20C22B3
:10B38C00900107E0FFEF6013900108E0FFE531D377
:10B39C009F40047F0122227F002222900108E0FFBF
:0DB3AC00E531C39F50047F0122227F002263
:10B278008F7B9000F7E0FF8F36AF7BEF3395E0FED2
:10B28800EF25E0FFEE33FE74012FF58274813EF561
:0FB2980083E493F508740193F509D229D20C22AF
:05001600C229C20C220A
:0C0096009000FEE0FF8F34D208C2092267
:05005600D208D20922CE
:10B75000900102E0FFEF60041294E8221269442293
:1094E800900245E0FFEF7016125349407290010553
:1094F800E0FF90000FEFF0900245E004F0229002A8
:1095080045E0FFEF64017028125349401C90000F9A
:10951800E0FFEF704AD25C90010FE0FF90000CEF83
:10952800F0900245E004F02222900245E4F0222265
:10953800900245E0FFEFB40221125349400B90011D
:109548000FE0FF90000CEFF02290000CE0FFEF70AE
:109558000EC25C900245E4F02222900245E4F0221B
:10694400900245E0FFEF704C900103E0FFEF6023FD
:10695400900104E0FFE532D39F4013900105E0FF6E
:1069640090000FEFF0900245E004F0228026C25C14
:10697400228021900104E0FFE532C39F501390016F
:1069840005E0FF90000FEFF09002457403F02280C1
:1069940003C25C22900245E0FFEF64017035900170
:1069A40004E0FFEF24FBFFE532D39F401F90000F6C
:1069B400E0FFEF6003026AA7D25C900106E0FF905B
:1069C4000010EFF0900245E004F02222900245E42A
:1069D400F02222900245E0FFEF6402702E90010441
:1069E400E0FFEF24FBFFE532D39F400B900106E06C
:1069F400FF900010EFF022900010E0FFEF60030220
:106A04006AA7C25C900245E4F02222900245E0FFAE
:106A1400EF64037043900104E0FF7E00EF2405FF60
:106A2400EE3400FEAD327C00C3ED9FEE6480F8ECE2
:106A3400648098501C90000FE0FFEF7066D25C9069
:106A44000106E0FF900010EFF0900245E004F02210
:106A540022900245E4F02222900245E0FFEF640414
:106A6400703C900104E0FF7E00EF2405FFEE34004B
:106A7400FEAD327C00C3ED9FEE6480F8EC64809838
:106A8400500B900106E0FF900010EFF022900010F0
:106A9400E0FFEF700EC25C900245E4F02222900207
:046AA40045E4F022B3
:1013E800202020464C4558204949492020202020CB
:1013F8000020202020202020202020202049444C8C
:1014080045004E4F204C5452204255532020494409
:101418004C45002054657374696E67204D6F646590
:101428002020200043726F73732042757379204D1A
:101438006F6465310043726F73732042757379204E
:101448004D6F6465320043726F7373204275737910
:10145800204D6F6465330043726F73732042757358
:1014680079204D6F6465340050726F6772616D6DDD
:10147800696E6757726F6E67004354435353203643
:10148800332E30202020202020435443535320362D
:10149800372E302020202020204354435353203619
:1014A800392E342020202020204354435353203702
:1014B800312E3920202020202043544353532037F5
:1014C800342E3420202020202043544353532037E7
:1014D800372E3020202020202043544353532037D8
:1014E800392E3720202020202043544353532038BE
:1014F800322E3520202020202043544353532038B7
:10150800352E3420202020202043544353532038A4
:10151800382E35202020202020435443535320398F
:10152800312E352020202020204354435353203986
:10153800342E382020202020204354435353203970
:10154800372E342020202020204354435353203169
:1015580030302E3020202020204354435353203154
:1015680030332E352020202020435443535320313C
:1015780030372E322020202020435443535320312B
:1015880031302E392020202020435443535320311A
:1015980031342E3820202020204354435353203107
:1015A80031382E38202020202043544353532031F3
:1015B80032332E30202020202043544353532031EF
:1015C80032372E33202020202043544353532031D8
:1015D80033312E38202020202043544353532031C8
:1015E80033362E35202020202043544353532031B6
:1015F80034312E33202020202043544353532031AC
:1016080034362E3220202020204354435353203197
:1016180035312E3420202020204354435353203189
:1016280035362E3720202020204354435353203171
:1016380035392E382020202020435443535320315D
:1016480036322E3220202020204354435353203159
:1016580036352E3520202020204354435353203143
:1016680036372E392020202020435443535320312D
:1016780037312E3320202020204354435353203128
:1016880037332E3820202020204354435353203111
:1016980037372E3320202020204354435353203102
:1016A80037392E39202020202043544353532031EA
:1016B80038332E35202020202043544353532031E3
:1016C80038362E32202020202043544353532031D3
:1016D80038392E39202020202043544353532031B9
:1016E80039322E38202020202043544353532031B0
:1016F80039362E362020202020435443535320319E
:1017080039392E352020202020435443535320328A
:1017180030332E3520202020204354435353203289
:1017280030362E3520202020204354435353203276
:1017380031302E3720202020204354435353203269
:1017480031382E3120202020204354435353203257
:1017580032352E3720202020204354435353203243
:1017680032392E3120202020204354435353203235
:1017780033332E3620202020204354435353203225
:1017880034312E3820202020204354435353203214
:1017980035302E3320202020204354435353203209
:1017A80035342E31202020202020202020202020E9
:1017B8002020202020202020204443532030303671
:1017C80020494E56203032312044435320303037A0
:1017D80020494E562032313420444353203031358D
:1017E80020494E562031343120444353203031377C
:1017F80020494E5620303530204443532030323172
:1018080020494E562030303620444353203032335E
:1018180020494E5620303437204443532030323547
:1018280020494E5620323434204443532030323637
:1018380020494E5620343634204443532030333127
:1018480020494E5620363237204443532030333215
:1018580020494E562030353120444353203033360A
:1018680020494E56203137322044435320303433F8
:1018780020494E56203434352044435320303437E1
:1018880020494E56203032332044435320303530DF
:1018980020494E56203031372044435320303531CB
:1018A80020494E56203033322044435320303533BC
:1018B80020494E56203435322044435320303534A5
:1018C80020494E5620343133204443532030363596
:1018D80020494E5620323731204443532030373187
:1018E80020494E5620333036204443532030373277
:1018F80020494E5620323435204443532030373364
:1019080020494E5620353036204443532030373452
:1019180020494E5620313734204443532031313446
:1019280020494E5620373132204443532031313537
:1019380020494E5620313532204443532031313628
:1019480020494E5620373534204443532031323213
:1019580020494E5620323235204443532031323507
:1019680020494E56203336352044435320313331F5
:1019780020494E56203336342044435320313332E5
:1019880020494E56203534362044435320313334D1
:1019980020494E56203232332044435320313431CB
:1019A80020494E56203031352044435320313433BA
:1019B80020494E56203431322044435320313435A7
:1019C80020494E5620323734204443532031353293
:1019D80020494E5620313135204443532031353586
:1019E80020494E5620373331204443532031353671
:1019F80020494E5620323635204443532031363262
:101A080020494E5620353033204443532031363553
:101A180020494E5620323531204443532031373245
:101A280020494E5620303336204443532031373432
:101A380020494E5620303734204443532032303525
:101A480020494E5620323633204443532032313217
:101A580020494E5620333536204443532032313402
:101A680020494E56203030372044435320323233F9
:101A780020494E56203133342044435320323235E6
:101A880020494E56203132322044435320323236D8
:101A980020494E56203431312044435320323433C8
:101AA80020494E56203335312044435320323434B4
:101AB80020494E56203032352044435320323435A5
:101AC80020494E5620303732204443532032343692
:101AD80020494E5620353233204443532032353185
:101AE80020494E5620313635204443532032353272
:101AF80020494E562034363220444353203235355F
:101B080020494E562034343620444353203236314F
:101B180020494E562037333220444353203236333F
:101B280020494E5620323035204443532032363532
:101B380020494E562031353620444353203236361C
:101B480020494E562034353420444353203237310F
:101B580020494E56203036352044435320323734FE
:101B680020494E56203134352044435320333036F3
:101B780020494E56203037312044435320333131E9
:101B880020494E56203636342044435320333135CD
:101B980020494E56203432332044435320333235C3
:101BA80020494E56203532362044435320333331B2
:101BB80020494E562034363520444353203333329F
:101BC80020494E562034353520444353203334338E
:101BD80020494E562035333220444353203334367F
:101BE80020494E5620363132204443532033353174
:101BF80020494E562032343320444353203335365F
:101C080020494E5620323132204443532033363453
:101C180020494E5620313331204443532033363542
:101C280020494E5620313235204443532033373132
:101C380020494E5620373334204443532034313121
:101C480020494E5620323236204443532034313214
:101C580020494E5620313433204443532034313305
:101C680020494E56203035342044435320343233F3
:101C780020494E56203331352044435320343331E4
:101C880020494E56203732332044435320343332D0
:101C980020494E56203531362044435320343435BC
:101CA80020494E56203034332044435320343436B0
:101CB80020494E562032353520444353203435329E
:101CC80020494E5620303533204443532034353490
:101CD80020494E5620323636204443532034353579
:101CE80020494E5620333332204443532034363271
:101CF80020494E562032353220444353203436345E
:101D080020494E562030323620444353203436354D
:101D180020494E562033333120444353203436363D
:101D280020494E562036363220444353203530332E
:101D380020494E5620313632204443532035303620
:101D480020494E562030373320444353203531360E
:101D580020494E5620343332204443532035323301
:101D680020494E56203234362044435320353236EB
:101D780020494E56203332352044435320353332E0
:101D880020494E56203334332044435320353436CB
:101D980020494E56203133322044435320353635BE
:101DA80020494E56203730332044435320363036AE
:101DB80020494E56203633312044435320363132A1
:101DC80020494E562033343620444353203632348B
:101DD80020494E562036333220444353203632377A
:101DE80020494E5620303331204443532036333176
:101DF80020494E562036303620444353203633325D
:101E080020494E5620363234204443532036353448
:101E180020494E5620373433204443532036363237
:101E280020494E5620343636204443532036363423
:101E380020494E5620333131204443532037303324
:101E480020494E5620353635204443532037313209
:101E580020494E5620313134204443532037323301
:101E680020494E56203433312044435320373331F0
:101E780020494E56203135352044435320373332DC
:101E880020494E56203236312044435320373334CC
:101E980020494E56203337312044435320373433BA
:101EA80020494E56203635342044435320373534A4
:101EB80020494E5620313136204284A4830124C360
:101EC800040274A344C282E364D4430381231463E9
:0F1ED80094B4C47D3D1D0D0585C5E5F5FD009550
:1078DA00900132E0FFB4010A9000A974FFF0E402BB
:1078EA0079A7EF640260030279AC12531B7880E631
:1078FA00600302799B30540302799B900238E0704E
:10790A0032D22D900119E024FF92499000A8E0FF9D
:10791A009001F9F0900117E09001FAF09001FBEF65
:10792A00F012586A9001FCEFF0128D0A9002387436
:10793A0002F02212848AEF64017050D22D9001F66F
:10794A00E0FF24E0F582E43401F583E09001F9F0E8
:10795A0074CB2FF582E43401F583E09001FAF090BC
:10796A0001F6E09001FBF01256B49001FCEFF090A2
:10797A0001F9E0245BF582E43401F583E024FF9207
:10798A0049128D0A900238E014F022900238E0146D
:10799A00F09000A8E09000A9F0900117E09000AAEA
:1079AA00F02290022DE0B40B0050469079BCF828E2
:1079BA0028730279DD0279E00279E30279E6027935
:1079CA00E90279EC0279FB0279EF0279F20279F5A0
:1079DA000279F80229A10271740272C702416B028C
:1079EA00992B0231C202B76F02B77E02B78D02B776
:0779FA009CE490022DF02235
:1029A1009000A8E0D3941440030231C190022EE0BC
:1029B100B40C0040030231BC9029C0F828287302EE
:1029C10029E40229FC022C3D022C84022CA1022CB8
:1029D100D2022DA8022E30022EC7022F06022FD0BE
:1029E1000230BD7BFF7A1379E812ABA67BFF7A1325
:1029F10079F912A5CC90022E022C39205523900290
:102A01006AE0701D204F127BFF7A1379E812ABA6A2
:102A11007BFF7A14790A12A5CC90026A7402F0C283
:102A21004F20A55C12531B900133E0600312532722
:102A3100900130E0900000F09000A8E0FF9000A924
:102A4100F0900117E0FE9000AAF090022E7405F0BC
:102A51009001F9EFF09001FAEEF09000A8E09001FA
:102A6100FBF01256B49001FCEFF0900119E024FF45
:102A71009249128D0AD22D7BFF7A14791B02ABA6E3
:102A810012A9A0EF6401706030465DC2469000A4B7
:102A9100E0FFC394155051745B2FF582E43401F5C6
:102AA10083E0FFA244E4336F703EA244924590005C
:102AB100A4E0900232F09000A5E0900233F0900083
:102AC100A3E0900234F012701D900234E0641F60A4
:102AD10017900232E0FF900233E0FD7C00128BC7B9
:102AE10090022D74020230E9C24612B528BF0117C7
:102AF10012531B900133E06003125327900130E021
:102B0100900000F0022EB1900134E0601C12A9A0E7
:102B1100EF6401600612B38CBF010E900111E078E1
:102B2100A4F690022E7409F02212A9A0EF6401709C
:102B310068302228C22290023A04F0D220854E4FFA
:102B4100E54F75F010A42481F9741435F0FA7BFF78
:102B510012ABA6AF4F1291B0C220802A302F3AC2D9
:102B61002F90023CE544F075F010A424C1F97417CC
:102B710035F0FA7BFF12ABA690023CE0FF128FFD0D
:102B810090023A7402F090022D7405F0E490022E46
:102B9100F0900111E078A4F622C222C22F78A6E6B5
:102BA10018467030900118E0FF6029760008A607EA
:102BB1009000A974FFF09000AAF012531B9001330A
:102BC100E06003125327900130E0900000F0900282
:102BD1002E02314B900123E0FF70030231C19000BE
:102BE10011E060030231C1900121E0FE6010700329
:102BF1000231C1900240E0640160030231C19000E2
:102C010011EFF0E4900240F012531B900133E060A9
:102C110003125327900130E0900000F09000A8E0EB
:102C21009000A9F09000AA74FDF0E490022EF090BB
:102C31000122E090022D60647401F022900000E016
:102C410060030231C13054030231C19000A8E0FF9A
:102C51009001F9F09001FA74FFF09001FBEFF09010
:102C610001FCF0900119E024FF9249128D0AD22D46
:102C71002036092037062038031270BF90022E74C7
:102C810003F0227880E660030231C130540302313F
:102C9100C190010CE0900001F090022E7404F0222A
:102CA100900001E060030231C1125321900133E031
:102CB100600312532DE490022EF090024004F020A4
:102CC100360C203709203806127D3A127D4C022D30
:102CD1009D30A503022D989000A8E09000A9F090E6
:102CE1000117E09000AAF012A9A0BF0105120096F9
:102CF10080031200567880E660030231C13054032C
:102D01000231C1900238E07034D22D900119E024D3
:102D1100FF92499000A8E0FF9001F9F0900117E0BF
:102D21009001FAF09001FBEFF012586A9001FCEF6C
:102D3100F0128D0A9002387402F00270BF12848A78
:102D4100EF6401704FD22D9001F6E0FF24E0F5828F
:102D5100E43401F583E09001F9F074CB2FF582E4BE
:102D61003401F583E09001FAF09001F6E09001FB67
:102D7100F01256B49001FCEFF09001F9E0245BF5FC
:102D810082E43401F583E024FF9249128D0A127026
:102D9100BF0231A00231A0E490022EF09000A9748C
:102DA100FFF09000AAF022900000E060030231C120
:102DB1003054030231C17880E660030231C19000D2
:102DC100A974FFF09000AAF0128622EF640160035B
:102DD100022EB89001F6E0FF24E0F582E43401F51B
:102DE10083E09001F9F074CB2FF582E43401F5838F
:102DF100E09001FAF09001F6E09001FBF012B6C20A
:102E01009001FCEFF09001F9E0245BF582E43401DC
:102E1100F583E024FF9249128D0AD22D2036092034
:102E210037062038031270BF90022E7407F0221269
:102E3100A9A0EF64017063304662C2469000A4E02D
:102E4100FFC394155056745B2FF582E43401F5836A
:102E5100E0FFA244E4336F7043A24492459000A482
:102E6100E0900232F09000A5E0900233F09000A3D0
:102E7100E0900234F012701D900234E0641F601C77
:102E8100900232E0FF900233E0FD7C00128BC7E438
:102E910090022EF090022D02314BC2467880E660FE
:102EA100030231C13054030231C112B528EF60076A
:102EB10090022E7406F02290010CE0900001F09037
:102EC100022E7408F022900001E060030231C11269
:102ED1005321900133E0600312532D90024074019D
:102EE100F0E490022EF09000A974FFF09000AAF097
:102EF1003036030231C13037030231C130380302A9
:102F010031C1027D4C12A9A0EF64017063304660AB
:102F1100C2469000A4E0FFC394155054745B2FF592
:102F210082E43401F583E0FFA244E4336F7041A2EF
:102F31004492459000A4E0900232F09000A5E09008
:102F41000233F09000A3E0900234F012701D900261
:102F510034E0641F601A900232E0FF900233E0FD1A
:102F61007C00128BC7E490022EF090022D02314BAF
:102F7100C24678A4E660030231C19000A8E0900047
:102F8100A9F09000AA74FDF0900134E0FF640160A3
:102F910004EFB4021512A9A0BF010F900112E09035
:102FA100000AF090022E740AF022900134E0FF64CE
:102FB100036004EFB4041512B38CBF010F9001122A
:102FC100E090000AF090022E740BF0220231BC1244
:102FD100A9A0BF0108900112E090000AF090000A38
:102FE100E0701B125321900118E0FF78A5760008CC
:102FF100A6079000A974FFF09000AA0230E99001A1
:1030010034E0B401097BFF7A14792C0230FA1253AF
:103011001B7BFF7A14793D12A5CC7880E660030210
:1030210031AD3054030231AD900238E07031D22D10
:10303100900119E024FF92499000A8E0FF9001F966
:10304100F0900117E09001FAF09001FBEFF01258B7
:103051006A9001FCEFF0128D0A90023802314B1296
:10306100848AEF6401704CD22D9001F6E0FF24E0D8
:10307100F582E43401F583E09001F9F074CB2FF58A
:1030810082E43401F583E09001FAF09001F6E090DA
:1030910001FBF01256B49001FCEFF09001F9E0242D
:1030A1005BF582E43401F583E024FF9249128D0A35
:1030B1000231A0900238E014F00231AD12B38CBF9E
:1030C1000108900112E090000AF090000AE0701CE3
:1030D100125321900118E0FF78A5760008A6079009
:1030E10000A974FFF09000AAF00231BC900134E015
:1030F100B403097BFF7A14794E02A5CC7BFF7A14C5
:10310100795F12A5CC12531B7880E660030231ADC2
:103111003054030231AD900238E07032D22D90016B
:1031210019E024FF92499000A8E0FF9001F9F09086
:103131000117E09001FAF09001FBEFF012586A904C
:1031410001FCEFF0128D0A9002387402F022128411
:103151008AEF64017050D22D9001F6E0FF24E0F572
:1031610082E43401F583E09001F9F074CB2FF5820C
:10317100E43401F583E09001FAF09001F6E090016A
:10318100FBF01256B49001FCEFF09001F9E0245BE2
:10319100F582E43401F583E024FF9249128D0A900F
:1031A1000238E014F022900238E014F09000A8E018
:1031B1009000A9F09000AA74FDF022E490022EF094
:0131C10022EB
:1071740090022EE0FF700F900000E060030272C6E0
:1071840090022F0272C0EF6401705F12A2B29002EB
:107194002FE0D39409400990010CE0900001802075
:1071A40090022FE0FF04F0743E2FF582E43401F5E1
:1071B40083E0900231F0E0FFB4260D9000017432B8
:1071C400F090022E7406F022EFB4240A900124E019
:1071D40075F006027279900231E0901EC19390021C
:1071E40031F05407900230F0807D90022EE064026A
:1071F400703912A2B2900124E0FF900002F09002D4
:1072040031E0FE30E709EF75F003A4900002F0EEE0
:1072140025E0900231F0900230E014F0900125E076
:10722400FF12B27890022E7403F02290022EE0B482
:10723400031E12A2B2900002E060030272C6900123
:1072440024E0900002F012001690022E7404F02242
:1072540090022EE06404702912A2B2900002E07041
:1072640061900230E0600790022E7402F0229001D7
:1072740024E075F003A4900002F090022E7405F04F
:107284002290022EE0B4050B12A2B2900002E0702C
:1072940031802A90022EE0B40628900001E070228A
:1072A400125321900133E0600312532D900118E032
:1072B400FF78A5760008A607E490022DF090022E30
:0372C40004F022B1
:1072C70090022EE0704F9000E5E0604212531B9051
:1072D7000133E06003125327900130E0900000F083
:1072E7009000E6E060229000E9E0B4300F9000E8FB
:1072F700E0B430089000E7E064306012206A0FD2F3
:107307006A90022D7407F02290022D027399900261
:107317002E7404F02290022EE0640170487880E613
:10732700600302740B30540302740B900232E09036
:1073370001F9F0900233E09001FAF09001FB741F1D
:10734700F01256B49001FCEFF0A2459249128D0A53
:10735700D22D2036092037062038031270BF90023D
:107367002E7402F02290022EE0640270297880E6E3
:10737700600302740B30540302740B90010CE0900D
:107387000001F0203609203706203803127D4C9083
:10739700022E7403F02290022EE0640370359000F1
:1073A70001E07060125321900133E0600312532D06
:1073B700900118E0FF78A5760008A607E490022D53
:1073C700F07BFF7A1379E812ABA67BFF7A1379F982
:1073D70002A5CC90022EE0D394034028E490022D1E
:1073E700F090022E04F07BFF7A1379E812ABA67BAC
:1073F700FF7A1379F912A5CC125321900133E0607B
:057407000312532D22C9
:10416B0090022EE0FF7017900232E09000A9F090C1
:10417B000233E09000AAF090022E7401F022EF645B
:10418B0001705A900000E06003024540A24592493D
:10419B00900232E09001F9F0900233E09001FAF0D6
:1041AB009000A8E09001FBF012586A9001FCEFF030
:1041BB00128D0AD22D2036092037062038031270B3
:1041CB00BF90010BE090000BF090010DE0900012FE
:1041DB00F09002387408F090022E02429190022E59
:1041EB00E06402702F126C0AEF600280467880E662
:1041FB0060030245403054030245407628D2549068
:10420B000238E014F0E060030245407402F09002C3
:10421B002E04F02290022EE0640360030242FB1294
:10422B006C0AEF6002800C90010DE0600D900012A3
:10423B00E0700790022E7404F0227880E66003028F
:10424B004540305403024540900238E0703CA24593
:10425B009249900232E09001F9F0900233E0900124
:10426B00FAF09000A8E09001FBF012586A9001FC64
:10427B00EFF0128D0AD22D20360920370620380395
:10428B001270BF9002387402F02212848AEF64011C
:10429B0070579001F6E0FF24E0F582E43401F583DA
:1042AB00E09001F9F074CB2FF582E43401F583E053
:1042BB009001FAF09001F6E09001FBF01256B490E9
:1042CB0001FCEFF09001F9E0245BF582E43401F599
:1042DB0083E024FF9249128D0AD22D20360B203712
:1042EB00082038051270BF8000900238E014F022CD
:1042FB0090022EE0640470342036092037062038F3
:10430B0003127D3A120056E4900239F09000E4E07B
:10431B006014900131E0FF12B24978A3761478A3B0
:10432B00E670FB12B80590022E7405F090022EE099
:10433B00640570457880E6704020543DA245924953
:10434B00900232E09001F9F0900233E09001FAF024
:10435B009001FB741FF012B6C29001FCEFF0128DAE
:10436B000A9002387403F0203609203706203803F0
:10437B001270BF90022E7406F090022EE0FF6406BE
:10438B0070297880E67024205421900238E0700F59
:10439B0090010CE0900001F090022E7407F022784F
:1043AB00807628D254900238E014F0EF6407600353
:1043BB00024540900134E0601F302209302F061275
:1043CB00B38CEF7013E490022DF090022EF090015D
:1043DB0011E078A4F602453412A9A0EF6401600342
:1043EB00024473204603024473C24612A9A0EF6431
:1043FB000170759000A4E0FFC39415506B745B2F94
:10440B00F582E43401F583E0FFA244E4336F705886
:10441B00A24492459000A4E0900232F09000A5E0F7
:10442B00900233F09000A3E0900234F0641F6038E8
:10443B00900232E0FFC39415502E745B2FF582E48B
:10444B003401F583E0FFA245E433B5071B9002323C
:10445B00E0FF900233E0FD7C00128BC790022D74BD
:10446B0002F0E490022EF0227880E6706920546608
:10447B00128622EF6401705E9001F6E0FF24E0F5F6
:10448B0082E43401F583E09001F9F074CB2FF582CF
:10449B00E43401F583E09001FAF09001F6E090012D
:1044AB00FBF01256B49001FCEFF09001F9E0245BA5
:1044BB00F582E43401F583E024FF9249128D0A90D2
:1044CB00022E7406F0E490022DF0203609203706F8
:1044DB002038031270BF900001E0705912532190E5
:1044EB000133E0600312532D2036092037062038A4
:1044FB0003127D4C9000A974FFF09000AAF090027B
:10450B00407401F0E490022DF090022E04F020365E
:10451B00182037152038127BFF7A1379E812ABA6D7
:10452B007BFF7A1379F912A5CC900118E0FF78A5DF
:06453B00760008A607222D
:10992B0090022EE0FF7017900000E07065F559F57E
:10993B005A9000F8E0F53490022E7401F022EFB447
:10994B00011D12A2B2D20B125D5F5013E4F559C286
:10995B000B90010CE0900001F090022E7402F0903D
:10996B00022EE06402702B12A2B2900001E0702272
:10997B00125321900133E0600312532D900118E034
:10998B00FF78A5760008A607E490022DF090022E32
:03999B0004F022B3
:1031C20090022EE060030232DC12A9A0EF640170CB
:1031D2005B304658C2469000A4E0FFC39415504CA1
:1031E200745B2FF582E43401F583E0FFA244E433FB
:1031F2006F7039A24492459000A4E0900232F090A0
:1032020000A5E0900233F09000A3E0900234F012A7
:10321200701D900234E0641F6012900232E0FF9051
:103222000233E0FD7C00128BC70234E9C24678A467
:10323200E6600302382E12A9A0EF64016003023295
:10324200C89000D9E07025125321900133E0600349
:1032520012532D900134E0B401109000A8E09000C8
:10326200A9F09000AA74FEF08070806612531B9041
:103272000133E06003125327900130E0900000F028
:103282009000A8E09000A9F09000AA74FEF09000CF
:10329200DBE0601A206A09D26A90022D7409F022DA
:1032A200125321900133E0600312532D80249001C8
:1032B2000DE0900012F0900110E090000DF09002ED
:1032C2002E7401F08014125321900133E060031236
:1032D200532DC220E490022DF02290022EE06401D0
:1032E2006003023377900000E060030233779002BC
:1032F2003AE064017036AF4F1295E3203671203701
:103302006E20386BE54F75F010A42481F9741435E2
:10331200F0FA7BFF12ABA6E54F75F010A42481F9F9
:10332200741435F0FA7BFF12A5CC804390023AE088
:103332006402704190023CE0FF12232420363020C8
:10334200372D20382A90023CE075F010A424C1F9F0
:10335200741735F0FA7BFF12ABA690023CE075F0D1
:1033620010A424C1F9741735F0FA7BFF12A5CC9092
:10337200022E02382890022EE0640270411267E0A9
:10338200EF6014127D3A90022E7403F09000D7E0A1
:10339200700302382E801E90010DE0602190001211
:1033A200E0701B127D3A90022E7403F09000D7E079
:1033B200700302382E90011DE0900004F02290026A
:1033C2002EE0640360030234F1900004E0704812BE
:1033D2007D4C120056E490023BF09000D7E060145E
:1033E200900131E0FF12B24978A3761978A3E67012
:1033F200FB12B8059000D8E0600F90011EE090002B
:103402000EF090022E7404F02290011FE09000034F
:10341200F012B7AB02350D12A9A0EF6401705A1277
:10342200B7AB30222CC22290023A7401F0C220853E
:103432004E4F203619203716203813E54F75F010FD
:10344200A42481F9741435F0FA7BFF12ABA602357D
:1034520041302F25C22F90023CE544F02036172040
:10346200371420381175F010A424C1F9741735F0FF
:10347200FA7BFF12ABA602356DC222C22F12A9A09F
:10348200EF6401706830466512B7ABC220C2469045
:1034920000A4E0FFC394155054745B2FF582E4340A
:1034A20001F583E0FFA244E4336F7041A2449245E8
:1034B2009000A4E0900232F09000A5E0900233F078
:1034C2009000A3E0900234F012701D900234E06488
:1034D2001F601A900232E0FF900233E0FD7C00127E
:1034E2008BC7E490022EF090022D023828C246903B
:1034F200022EE0640460030235F990000EE07011C0
:1035020012B7AB90011FE0900003F090022E023739
:10351200AA12A9A0EF6401706B12B7AB302230C2BD
:103522002290023A7401F0854E4FC220E54F75F0A9
:1035320010A42481F9741435F0FA7BFF12ABA6AF04
:103542004F1291B0E490022EF090022D0237AA3071
:103552002F32C22F90023CE544F075F010A424C132
:10356200F9741735F0FA7BFF12ABA690023CE0FF2C
:10357200128FFD90023A7402F0E490022EF0900253
:103582002D0237AAC222C22F12A9A0EF64017065D0
:1035920030466212B7ABC220C2469000A4E0FFC31D
:1035A20094155051745B2FF582E43401F583E0FFEA
:1035B200A244E4336F703EA24492459000A4E0908E
:1035C2000232F09000A5E0900233F09000A3E09068
:1035D2000234F012701D900234E0641F60179002F2
:1035E20032E0FF900233E0FD7C00128BC790022D87
:1035F2007402023676C24690022EE064056003022F
:1036020036F3900003E0700790022E7406F0221247
:10361200A9A0EF6401706430222BC22290023A0406
:10362200F0854E4FC220E54F75F010A42481F97445
:103632001435F0FA7BFF12ABA6AF4F1291B0900295
:103642002D7405802F302F33C22F90023CE544F0B9
:1036520075F010A424C1F9741735F0FA7BFF12AB90
:10366200A690023CE0FF128FFD90023A7402F090A5
:10367200022D7405F0E490022EF022C222C22F1213
:10368200A9A0EF6401706830466512B7ABC220C2D0
:10369200469000A4E0FFC394155054745B2FF5824A
:1036A200E43401F583E0FFA244E4336F7041A244A5
:1036B20092459000A4E0900232F09000A5E09002C2
:1036C20033F09000A3E0900234F012701D900234A7
:1036D200E0641F601A900232E0FF900233E0FD7C4A
:1036E20000128BC7E490022EF090022D023828C2FD
:1036F2004690022EE06406600302382E900001E03C
:10370200703D125321900133E0600312532D7BFF71
:103712007A1379E812ABA67BFF7A1379F912A5CC5A
:10372200900118E0FF78A5760008A6079002407481
:1037320001F0C220E490022DF090022E04F0221239
:10374200A9A0EF6401706530222CC22290023A04D3
:10375200F0854E4FE54F75F010A42481F9741435AD
:10376200F0FA7BFF12ABA6AF4F1291B0E490022E9B
:10377200F090022D8032302F33C22F90023CE5446C
:10378200F075F010A424C1F9741735F0FA7BFF121A
:10379200ABA690023CE0FF128FFD90023A7402F059
:1037A200E490022EF090022D7405F022C222C22F64
:1037B20012A9A0EF6401707230466F12B7ABC2203B
:1037C200C2469000A4E0FFC39415505E745B2FF5CF
:1037D20082E43401F583E0FFA244E4336F704BA22C
:1037E2004492459000A4E0900232F09000A5E0904F
:1037F2000233F09000A3E0900234F0203609203723
:103802000620380312701D900234E0641F601B9082
:103812000232E0FF900233E0FD7C00128BC7E4909D
:0D382200022EF090022D7402F022C2462208
:0FB76F007BFF7A14797012ABA6E490022DF022C2
:0FB77E007BFF7A14797012ABA6E490022DF022B3
:0FB78D007BFF7A14797012ABA6E490022DF022A4
:0FB79C007BFF7A14797012ABA6E490022DF02295
:1045410043544353532036332E3020202020202043
:1045510043544353532036372E302020202020202F
:1045610043544353532036392E3420202020202019
:1045710043544353532037312E392020202020200B
:1045810043544353532037342E34202020202020FD
:1045910043544353532037372E30202020202020EE
:1045A10043544353532037392E37202020202020D5
:1045B10043544353532038322E35202020202020CD
:1045C10043544353532038352E34202020202020BB
:1045D10043544353532038382E35202020202020A7
:1045E10043544353532039312E352020202020209D
:1045F10043544353532039342E3820202020202087
:1046010043544353532039372E3420202020202077
:104611004354435353203130302E3020202020206A
:104621004354435353203130332E35202020202052
:104631004354435353203130372E32202020202041
:104641004354435353203131302E39202020202030
:104651004354435353203131342E3820202020201D
:104661004354435353203131382E38202020202009
:104671004354435353203132332E30202020202005
:104681004354435353203132372E332020202020EE
:104691004354435353203133312E382020202020DE
:1046A1004354435353203133362E352020202020CC
:1046B1004354435353203134312E332020202020C2
:1046C1004354435353203134362E322020202020AE
:1046D1004354435353203135312E342020202020A0
:1046E1004354435353203135362E37202020202088
:1046F1004354435353203135392E38202020202074
:104701004354435353203136322E3220202020206F
:104711004354435353203136352E35202020202059
:104721004354435353203136372E39202020202043
:104731004354435353203137312E3320202020203E
:104741004354435353203137332E38202020202027
:104751004354435353203137372E33202020202018
:104761004354435353203137392E39202020202000
:104771004354435353203138332E352020202020F9
:104781004354435353203138362E322020202020E9
:104791004354435353203138392E392020202020CF
:1047A1004354435353203139322E382020202020C6
:1047B1004354435353203139362E362020202020B4
:1047C1004354435353203139392E352020202020A2
:1047D1004354435353203230332E352020202020A0
:1047E1004354435353203230362E3520202020208D
:1047F1004354435353203231302E37202020202080
:104801004354435353203231382E3120202020206D
:104811004354435353203232352E37202020202059
:104821004354435353203232392E3120202020204B
:104831004354435353203233332E3620202020203B
:104841004354435353203234312E3820202020202A
:104851004354435353203235302E3320202020201F
:104861004354435353203235342E3120202020200D
:104871002020202020202020202020202020202037
:1048810044313233343536373839302A23414243C3
:107B250075840F1254F912B4659000A8E0FF600542
:107B3500D3941440069000A87401F0128A7612A01E
:107B4500EB12A14712B35F125343129F73125321D5
:107B5500123CE2900118E0FF78A5760008A607E43C
:107B650090018BF090022EF090022DF0900239F0EA
:107B750090023EF0129D71E4900241F0900011F0E8
:107B8500125333D2ACD2A830311D12B4DB12B46516
:107B9500128A7612A0EB12A14712B35FC236C23722
:107BA500C23812382F80E0120056127D4C20A32CCB
:107BB500303F12C23F787EE6540F90488193900182
:107BC5008AF01295683040E5C240787CE6540F9003
:107BD500488193900189F012965E80D120A4051208
:107BE5009EA980F8128863304126C24112B4DB1287
:107BF500B465128A7612A0EB12A14712B35FC236A2
:107C0500C237C238129F73E490022DF090022EF015
:107C1500203606203703303805127D5E80F243E7B3
:107C250040900013E0700E305508129F1012B502F7
:107C350080031290901278DA12497512768512B780
:037C4500508099D3
:105A0A008DB7948A98419BDC9F3AA27EA5A9A8BA31
:105A1A00ABB1AEA5B150B40DB614B800BA6FBCD6CE
:105A2A00BF14C148C365C577C74FC95FCB41CD0B0A
:105A3A00CEC1D072D20DD2F2D39CD47FD51ED5F866
:105A4A00D693D764D7FAD8C3D955DA16DAA8DB6160
:105A5A00DBE9DC9FDD22DDD4DEFDE019E093E12EF7
:105A6A00E239E33CE3AA0000000000000000000065
:105A7A00000000000000000000000000000000001C
:105A8A00000000000000000000000000000000000C
:105A9A0000000000000000010000000000010000FA
:105AAA0000000001000000000000000100000000EA
:105ABA0000010000000000010000000000010000D9
:105ACA0000000001000000000001000000000001C9
:105ADA0000000000000100000000000100000001B9
:105AEA0000010000000100010000000100010000A7
:105AFA000001000100000000000100010000000197
:105B0A000001000000010001000000010001000086
:105B1A000001000100000001000100000001000175
:105B2A000000000100010000000100010000000166
:105B3A000001000000010001000000010001000056
:105B4A000001000100000001000100000001000145
:105B5A000000000100010000000100010000000136
:105B6A000001000000010001000000010001000026
:105B7A000001000100000001000100010001000114
:105B8A000001000100010001000100010001000103
:0E5B9A000001000100010001000100010001F6
:1095E300C22BC22DD2B3D2B275F006EFA42470F50C
:1095F30082E5F0345AF583E493FC740193FDEC4D5A
:1096030024FF92B075F006EFA42472F582E5F034DE
:109613005AF583E493FC740193FDEC4D24FF92B758
:1096230075F006EFA42474F582E5F0345AF583E46B
:1096330093FC740193FDEC4D24FF92B5EF25E024D8
:109643000AF582E4345AF583E493F52E740193F515
:0B9653002FD22CE4F584D28CD2A92287
:0EB7AB00C22BC22DC22CE4F584C28CC2A9228E
:104EC50020504C55472050484F4E454C494E4520A3
:104ED50000554E504C55472050484F4E454C494E75
:104EE5004500504C5547494E2050484F4E454C497A
:104EF5004E450044313233343536373839302A237C
:104F050041424302AB055508000AAB0D551000128E
:104F1500AB155518001AAB1D55200022AB25552899
:104F2500002AAB2D55300032AA3555202054455363
:104F35005420524F5554494E452020202056455265
:104F450053494F4E20312E302020202054455354B4
:104F5500494E4720454550524F4D2020205445533A
:104F650054494E4720564F494345202054455354F4
:104F7500494E472044544D46203120205445535432
:104F8500494E472044544D46203220202054455355
:104F950054494E4720525332333220202054455332
:104FA50054494E472052533438352020202054454B
:104FB5005354494E472050545420202054455354AF
:104FC500204155582052454C4159202054455354B1
:104FD5002043542052454C415920202054455349E3
:104FE5004E472052494E47494E4720202020202039
:104FF50020202020202020202020202054455354EC
:10500500204C494E45204C4F4F5020544553542079
:105015004C494E452053454E53452B54455354203A
:105025004C494E452053454E53452D544553542028
:105035004C494E4520494E2055534520544553541F
:1050450020494E50555420564F4C542054455354E6
:10505500204C494E452052454C4159544553542006
:105065005A45524F2043524F5353205445535449A8
:105075004E4720535155454C434820202054455315
:1050850054494E472048504620202020544553542B
:105095002054454C434F20564F58202054455354D7
:1050A50020524144494F20564F582020202020208F
:1050B50020202020202020202020202020202020EB
:1050C50020202020202020202020202020202020DB
:1050D500202020202020202020202020544553540B
:1050E50020434F4D504C45544544202020205445E5
:0B50F5005354204641494C4544202004
:10382F007BFF7A4F793012ABA67BFF7A4F7940122C
:10383F00A5CC12B7F17BFF7A4F795012ABA6127D50
:10384F004C12B7F1E4FFFE12758D900170EFF07D11
:10385F00AAE4FFFE12754CE4FFFE12758DEF64AA09
:10386F00600C7BFF7A5079F012A5CC1200717D5558
:10387F00E4FFFE12754CE4FFFE12758DEF64556088
:10388F000C7BFF7A5079F012A5CC12007190017069
:10389F00E0FDE4FFFE12754C7BFF7A5079E012AB2E
:1038AF00A612B7F17BFF7A4F796012ABA612533B8A
:1038BF0012B7DBE4F559755A01789E7614125D56EE
:1038CF00789EE670FB125D4D12B805E4F559755AF6
:1038DF0001789E7605789EE670FBD202D20B125DC0
:1038EF0044C202C20B7BFF7A5079E012ABA612B72B
:1038FF00F17BFF7A4F797012ABA6127D4C12B7F1A4
:10390F00C2277F3112B658789E761E789EE670FBDE
:10391F0012B80C3027FD787EE6547F904EF8937BDB
:10392F00FFB4310C7A5079E012ABA612B7F1800ACE
:10393F007A5079F012A5CC1200717BFF7A4F798003
:10394F0012ABA6127D4C12B7F17F3112B64112B7EE
:10395F00FB12B80C3025FD787CE6547F904EF8931F
:10396F007BFFB4310C7A5079E012ABA612B7F1801D
:10397F000A7A5079F012A5CC1200717BFF7A4F7939
:10398F009012ABA6127D4C12B7F1E4F584759850E6
:10399F00C299C2987599433098FDE4F584E599640E
:1039AF0043600C7BFF7A5079F012A5CC1200717B2B
:1039BF00FF7A5079E012ABA612B7F17BFF7A4F79FD
:1039CF00A012ABA6127D4C12B7F1125346E4F58448
:1039DF00759850C299C2987599433099FD7BFF7ABB
:1039EF005079E012ABA612B7F17BFF7A4F79B01284
:1039FF00ABA6127D4C12B7F112531B12B7FBE53277
:103A0F00D39432400C7BFF7A5079F012A5CC120080
:103A1F007112532112B7FBE532C394AA500C7BFFEE
:103A2F007A5079F012A5CC1200717BFF7A5079E0B1
:103A3F0012ABA612B7F17BFF7A4F79C012ABA61269
:103A4F007D4C12B7F112532712B7FBE531D3940A0D
:103A5F00400C7BFF7A5079F012A5CC1200711253F3
:103A6F002D12B7FBE531C394AA500C7BFF7A507926
:103A7F00F012A5CC1200717BFF7A5079E012ABA641
:103A8F0012B7F17BFF7A4F79E012ABA6127D4C1281
:103A9F00B7F112535E40FB7BFF7A5079E012ABA671
:103AAF0012B7F17BFF7A50790012ABA6127D4C1240
:103ABF00B7F112533312B7FB12536A501A125370E5
:103ACF0040157BFF7A50791012ABA612536A40FB58
:103ADF0012537050F6801D12536A50DC125370400F
:103AEF00D77BFF7A50792012ABA612536A40FB1294
:103AFF00537050F67BFF7A5079E012ABA612B7F1F4
:103B0F0012533B7BFF7A50793012ABA6127D4C12C9
:103B1F00B7F112533B12536450107BFF7A4E79C5A5
:103B2F0012A5CC12536440FB800E7BFF7A4E79D6E0
:103B3F0012A5CC12536450FB127D4C7BFF7A507947
:103B4F00E012ABA612B7F112533B7BFF7A507940CC
:103B5F0012ABA6127D4C12B7F1E530C3940A4007A1
:103B6F00E530D3943C400C7BFF7A5079F012A5CC12
:103B7F001200717BFF7A5079E012ABA612B7F17B7E
:103B8F00FF7A50795012ABA6127D4C12B7F1125337
:103B9F003312B7FB125355400B7BFF7A4E79E71266
:103BAF00ABA680F07BFF7A5079E012ABA612B7F18B
:103BBF0012533B7BFF7A50796012ABA6127D4C12E9
:103BCF00B7F112B7C512535B40FB12535B50FB1298
:103BDF00535B40FB7BFF7A5079E012ABA612B7F133
:103BEF0012B8057BFF7A50797012ABA6127D4C127A
:103BFF00B7F1125349400B12531B12532112534961
:103C0F0050F57BFF7A5079E012ABA612B7F17BFF2C
:103C1F007A5079A012ABA6127D4C12B7F112B7D021
:103C2F0012534F50FB12B8057BFF7A5079E012AB5D
:103C3F00A612B7F17BFF7A50798012ABA6127D4C9A
:103C4F0012B7F112B7C512B6F3904F0A12B6EA9037
:103C5F004F0C12B6EA904F0E12B6EA904F1012B6F2
:103C6F00EA904F1212B6EA904F1412B6EA904F161E
:103C7F0012B6EA904F1812B6EA904F1A12B6EA909F
:103C8F004F1C12B6EA904F1E12B6EA904F2012B692
:103C9F00EA904F2212B6EA904F2412B6EA904F26BE
:103CAF0012B6EA904F2812B6EA904F2A12B6EA904F
:103CBF004F2C12B6EA904F2EE493F508740193F54A
:103CCF000912B8057BFF7A5079E012ABA612B7F153
:033CDF00023C5252
:0AB7F100789E760A789EE670FB222F
:0AB7FB00789E7602789EE670FB222D
:09B6EA00E493F508740193F509DD
:0AB6F300789E7605789EE670FB2233
:0200710080FE0F
:0300A30002A95D52
:10A95D00C0E0C0F0C083C082C0D075D000C000C0C0
:10A96D0001C002C003C004C005C006C007205505C4
:10A97D001282E4800312A4B6D007D006D005D0040D
:10A98D00D003D002D001D000D0D0D082D083D0F06F
:03A99D00D0E032D5
:03009300029C3399
:099C3300C0E0C0D075D000C007EC
:109C3C00AF84758402E543700885BE3375BB07801D
:109C4C0032E543B4010885BE3075BB048025E5437D
:109C5C00B4020885BE3375BB068018E543B403080F
:109C6C0085BE3175BB04800BE543B4040A85BE3355
:109C7C0075BB0505438010E543B4050885BE3275F8
:0B9C8C00BB048000754300C2ED8F8414
:079C9700D007D0D0D0E0326D
:0300830002ABDEEF
:10ABDE00C0E0C0F0C083C082C0D075D000C000C03D
:10ABEE0001C002C003C004C005C006C007C2CF1218
:10ABFE00219DD007D006D005D004D003D002D001BD
:0DAC0E00D000D0D0D082D083D0F0D0E03282
:03007B0002A032AE
:10A03200C0E0C0F0C083C082C0D075D000C000C0F4
:10A0420001C002C003C004C005C006C00720240F1F
:10A0520085BF4085BE3FD22475BB01C2ED8013850A
:10A06200BF3E85BE3DC22430580312812B75BB0012
:10A07200C2EDD007D006D005D004D003D002D00163
:0DA08200D000D0D0D082D083D0F0D0E0321A
:03007300028F6990
:108F6900C0E0C0F0C083C082C0D075D000C000C0CE
:108F790001C002C003C004C005C006C007C2CF7843
:108F89009AE6600116302E27124BD8C22ED55C0501
:108F9900755C0A055BD51B09751B0A758401438835
:108FA90020D51C19751C60758402438820800ED257
:108FB9002E789B16E670067604F584D28B3055051B
:108FC900129DDA800312A36112923D1297C975842A
:108FD90001438810758400D2ECD007D006D005D0A3
:108FE90004D003D002D001D000D0D0D082D083D019
:048FF900F0D0E032A2
:03006B000287A366
:1087A300C0E0C0F0C083C082C0D075D000C000C09C
:0D87B30001C002C003C004C005C006C0071D
:1087C00085841620261875840F30DF3875840FE5F0
:1087D000E8540F787CF6D226787D76C88026787D9E
:1087E00016E6700E75840FE5E8540F787CF6E644C3
:1087F00080F675840F20DF0CC226D225D240D262CB
:10880000D25FD26820281630F833E5E854F0FFC470
:10881000540F787EF6D228787F76C88020787F162D
:10882000E6700FE5E854F0FFC4540F787EF6E64496
:1088300080F620F808C228D227D23FD26112740CE9
:08884000758402C28D851684C7
:10884800D007D006D005D004D003D002D001D00084
:0B885800D0D0D082D083D0F0D0E0322E
:03005B0002A1A35C
:10A1A300C0E0C0F0C083C082C0D075D000C000C082
:10A1B30001C002C003C004C005C006C0071248AAFC
:10A1C300789CE6600116E5416002154190000CE0C1
:10A1D300600214F0900247E0600214F0758401C23B
:10A1E3008DD007D006D005D004D003D002D001D043
:0CA1F30000D0D0D082D083D0F0D0E03279
:0300530002A80AF6
:10A80A00C0E0C0F0C083C082C0D075D000C000C014
:10A81A0001C002C003C004C005C006C007C28C3014
:10A82A005A04C25A8005D25A124CF7D007D006D021
:10A83A0005D004D003D002D001D000D0D0D082D02D
:06A84A0083D0F0D0E032E3
:03002B0002000FC1
:03000F00C2CF322B
:03001B0002006E72
:03006E00C28F320C
:0300130002ADBC7F
:10ADBC00C0E0C0F0C083C082C0D075D000C000C05D
:10ADCC0001C002C003C004C005C006C007121EE7C4
:10ADDC00D007D006D005D004D003D002D001D000CB
:0BADEC00D0D0D082D083D0F0D0E03275
:10AA6300191823A01296203D129623A0129627634D
:10AA73001488203D148823A01488276316B8203D2A
:10AA830016B823A016B827631918203D1918276391
:10AA930012962B8C14882B8C16B82B8C19182B8C94
:0BB7DB0075081575095ED229D2032203
:0BB7E60075081575095ED229D20C22EF
:07B80500C229C203C20C229C
:10B64100E4F512F513F514F5159000F3E0F5351254
:07B651006EC5D22AD20422CB
:10B65800E4F512F513F514F5159000F4E0F535123C
:07B668006EC5D22AD20D22AB
:106EC500EF127F386FC0236FAF2A6EFD306F0F3121
:106ED5006F21326F33336F45346F57356F69366FB6
:106EE5007B376F8D386F9E396FD1416FE2426FF3FB
:106EF500437004440000701C90AA63E493F50D747C
:106F05000193F50E90AA6502701390AA67E493F5B4
:106F15000D740193F50E90AA6902701390AA6BE4A3
